:020000040800F2
:10000000B803002099360008BB110008BD11000894
:10001000C1110008C5110008C91100080000000046
:10002000000000000000000000000000CD110008EA
:10003000CF11000800000000D1110008D311000802
:10004000AF360008AF360008AF360008AF360008FC
:10005000AF360008AF360008AF360008AF360008EC
:10006000AF360008AF360008AF360008AF360008DC
:10007000AF360008AF360008AF360008AF360008CC
:10008000AF360008AF360008AF360008AF360008BC
:10009000AF360008AF360008AF360008AF360008AC
:1000A000AF360008AF360008AF360008AF3600089C
:1000B000AF360008AF360008AF360008AF3600088C
:1000C000AF360008AF360008AF360008AF3600087C
:1000D000AF360008AF360008AF360008AF3600086C
:1000E000AF360008AF360008AF36000800F002F85F
:1000F00000F044F80AA090E8000C82448344AAF17E
:100100000107DA4501D100F039F8AFF2090EBAE87B
:100110000F0013F0010F18BFFB1A43F0010318473B
:10012000B86B0000D86B0000103A24BF78C878C1C3
:10013000FAD8520724BF30C830C144BF04680C60ED
:10014000704700000023002400250026103A28BF35
:1001500078C1FBD8520728BF30C148BF0B60704739
:10016000782904F0E180732904F0B98200207047F7
:100170001FB504F0B6F91FBD10B510BD04F0B3FAF9
:100180001146FFF7F5FF00F0F7FF04F0D1FA03B4D2
:10019000FFF7F2FF03BC04F0D7FA00000B49D1F8D7
:1001A00000C04A685CF8043B1068184442F8040B2D
:1001B0008C4528BFA1F1DC0C8A4228BFA1F1DC02EA
:1001C000C1F800C04A6020F0004070475001002094
:1001D00070B505460E4614463146284602F0C4FC6A
:1001E000204602F046FC70BD2DE9F05F04460D4646
:1001F00016461F46301B401C1FFA80FA781B401C15
:100200001FFA80FB3B4632462946204602F082FC1C
:100210004FF000080FE04FF0000906E00A9802F0E6
:1002200028FC09F101001FFA80F9D145F6DB08F13D
:1002300001001FFA80F8D845EDDBFD484088401EDC
:1002400083B2FB480088401E82B20021084602F0BB
:1002500061FCBDE8F09F2DE9FF4F85B081468A46DD
:100260000020049003900798A0EB09050898A0EBE4
:100270000A06CDF80890CDF804A0002D01DD012775
:1002800005E00DB9002702E04FF0FF376D42002E68
:1002900002DD4FF0010806E016B94FF0000802E059
:1002A0004FF0FF387642B54201DD2C4600E034467F
:1002B0004FF0000B21E0019A91B2029A90B202F045
:1002C0005DFC0498284404900398304403900498FB
:1002D000A04205DD0498001B049002983844029067
:1002E0000398A04205DD0398001B03900198404449
:1002F00001900BF101001FFA80FB601C8345DADDE1
:1003000009B0BDE8F08F2DE9F04104460D461646D0
:100310001F46DDF81880EA1991B2A21990B2424640
:10032000FFF756FFEA1991B2A21B90B24246FFF7BF
:100330004FFFEA1B91B2A21990B24246FFF748FF65
:10034000EA1B91B2A21B90B24246FFF741FFAA19E5
:1003500091B2E21990B24246FFF73AFFAA1991B260
:10036000E21B90B24246FFF733FFAA1B91B2E2199B
:1003700090B24246FFF72CFFAA1B91B2E21B90B24B
:100380004246FFF725FFBDE8F0812DE9FF4F81B020
:10039000824617469846DDF838B0002445464FEAB5
:1003A0004800C0F10306BBF1000F1FD01BE0A146BF
:1003B00008E04B462246009750460299FFF7A3FFFC
:1003C00009F10109A945F4DD002E04DA042000FB3F
:1003D0000460861D06E0601B042101FB006000F143
:1003E0000A066D1E641CAC42E1DD18E015E02B46E8
:1003F0002246009750460299FFF785FF002E04DA47
:10040000042000FB0460861D06E0601B042101FB44
:10041000006000F10A066D1E641CAC42E7DD05B009
:10042000BDE8F08F2DE9FF4F85B081460020049094
:1004300083460798A0EB090506990898461ACDF857
:100440000C9006980290002D01DD012705E00DB902
:10045000002702E04FF0FF376D42002E02DD4FF023
:10046000010806E016B94FF0000802E04FF0FF382F
:100470007642B54201DD2C4600E034464FF0000ADA
:100480001FE001200090DDE91232DDE90210FFF7E4
:100490007CFF049828440490B3440498A04205DDEE
:1004A0000498001B0490039838440390A34504DD8E
:1004B000ABEB040B0298404402900AF101001FFAD2
:1004C00080FA601C8245DCDD09B0BDE8F08F2DE9C3
:1004D000F04104460D4616461F462B463246294635
:1004E0002046FFF7B8FE3B46224629462046FFF746
:1004F000B2FE3B46324639462046FFF7ACFE3B464D
:10050000324629463046FFF7A6FEBDE8F081F8B531
:1005100004460D4616461F46464800883B4632466E
:10052000294600902046FFF75FFEF8BD2DE9F84F01
:1005300006460F4691469846C9F101000FFA80FA27
:100540004FF0010B4FEA4900404200B200900024F6
:100550004D4652E0BAF1000F09DB681E85B20098E3
:10056000801C00B20090009850440FFA80FA601C82
:1005700084B20BF102000FFA80FB0AEB0B000FFABA
:1005800080FA08F0040058B17A1991B2321990B289
:1005900002F0F4FA3A1991B2721990B202F0EEFA3E
:1005A00008F0020058B17A1B91B2321990B202F0F1
:1005B000E5FA3A1B91B2721990B202F0DFFA08F034
:1005C000080058B13A1991B2721B90B202F0D6FAF3
:1005D0007A1991B2321B90B202F0D0FA08F0010001
:1005E00058B13A1B91B2721B90B202F0C7FA7A1B53
:1005F00091B2321B90B202F0C1FAAC42AADBBDE864
:10060000F88F2DE9FC5F06460F4690469A46DDF8C6
:100610003090C8F101000FFA80FB012001904FEAF1
:100620004800404200B200900024454675E00000BA
:10063000640000202E000020BBF1000F09DB681EC3
:1006400085B20098801C00B20090009858440FFAC0
:1006500080FB601C84B20198801C00B2019001985C
:1006600058440FFA80FB0AF0010048B307EB050C71
:100670000CF1010CCC441FFA8CF306EB040C1FFAAE
:100680008CF2A7EB050C1FFA8CF106EB040C1FFA99
:100690008CF0FFF7E0FD07EB040C0CF1010CCC44EF
:1006A0001FFA8CF306EB050C1FFA8CF2A7EB040C77
:1006B0001FFA8CF106EB050C1FFA8CF0FFF7CBFD4F
:1006C0000AF0020048B307EB050C0CF1010CCC4416
:1006D0001FFA8CF3A6EB040C1FFA8CF2A7EB050CA7
:1006E0001FFA8CF1A6EB040C1FFA8CF0FFF7B3FD98
:1006F00007EB040C0CF1010CCC441FFA8CF3A6EBB5
:10070000050C1FFA8CF2A7EB040C1FFA8CF1A6EB78
:10071000050C1FFA8CF0FFF79EFDAC428CDBBDE8A8
:10072000FC9F2DE9F04105460E4617469846069C6B
:10073000391B8AB2291988B233463146FFF78BFD3F
:10074000A8EB040083B2301981B22A462846FFF78D
:1007500082FD391B8AB2291988B243464146FFF708
:100760007AFDA8EB040083B2301981B23A463846CC
:10077000FFF771FD321991B22A1990B20123224676
:10078000FFF7D4FE321991B23A1B90B202232246EF
:10079000FFF7CCFEA8EB040291B23A1B90B20423FF
:1007A0002246FFF7C3FEA8EB040291B22A1990B2C9
:1007B00008232246FFF7BAFEBDE8F0812DE9F84391
:1007C00007460D4690461E46089CFA480088711C54
:1007D0008BB2A8EB04018AB23919009088B229467D
:1007E000FFF702FD701B401C022101FB1400401E9C
:1007F00080B22A1991B2A8EB0402009090B20123B2
:100800002246FFF7FEFE701B401C022101FB140074
:10081000401E80B22A1991B23A19009090B2022378
:100820002246FFF7EEFEBDE8F8832DE9F0470446C7
:100830000D4616461F46DDE908893B4632462946E5
:100840002046FFF708FD4B46424639463046FFF743
:1008500002FD2B46224649464046FFF7FCFCBDE818
:10086000F08702880B8803800A8070472DE9FF4FCC
:1008700085B000260027BDF81800BDF8201088427A
:1008800007DD08A906A8FFF7ECFF07A905A8FFF7F1
:10089000E8FFBDF82000BDF84C10884207DD08A92C
:1008A00013A8FFF7DEFF07A912A8FFF7DAFFBDF8CC
:1008B0001800BDF82010884207DD08A906A8FFF738
:1008C000D0FF07A905A8FFF7CCFFBDF81800BDF8B9
:1008D0004C10884238D1BDF8140003900490BDF844
:1008E0001C00BDF81010884203DABDF81C0004900B
:1008F00008E0BDF81C00BDF80C10884202DDBDF810
:100900001C000390BDF84800BDF81010884203DABF
:10091000BDF84800049008E0BDF84800BDF80C1090
:10092000884202DDBDF848000390A248008800908C
:10093000BDF81830BDF80C201946BDF81000FFF7BF
:1009400053FC09B0BDE8F08FBDF81C00BDF81410D1
:10095000A0EB010BBDF82000BDF81810401A029062
:10096000BDF84800BDF81410451ABDF84C00BDF89C
:100970001810A0EB0109BDF84800BDF81C10A0EB51
:10098000010ABDF84C00BDF82010401A0190BDF8D6
:100990002000BDF84C10884202D1BDF8208004E050
:1009A000BDF82000401E1FFA80F8BDF8184027E06F
:1009B000029896FBF0F0BDF81410084480B2049041
:1009C00097FBF9F0BDF81410084480B203905E4420
:1009D0002F44BDF81000BDF80C10884203DD03A9B8
:1009E00004A8FFF73EFF7348008823460090BDF837
:1009F0000C202146BDF81000FFF7F6FB601C84B206
:100A00004445D5DDBDF82000201A00FB0AF6BDF8EC
:100A10001800201A00FB05F727E0019896FBF0F07C
:100A2000BDF81C10084480B2049097FBF9F0BDF8A3
:100A30001410084480B2039056442F44BDF81000AF
:100A4000BDF80C10884203DD03A904A8FFF709FFD5
:100A50005848008823460090BDF80C202146BDF878
:100A60001000FFF7C1FB601C84B2BDF84C0084424B
:100A7000D3DD00BF65E72DE9FF4F83B081468A468D
:100A80009346DDE910644B4800880290A6F12000EF
:100A9000C6B204EBD47009EB6000401E82B20AEBD0
:100AA0000400401E83B251464846019402F032F8D9
:100AB000129850BB002525E00C2C07D106EB460010
:100AC0003D4901EB800010F8058004E03B4800EB55
:100AD000061010F8058000270DE008F0010018B19D
:100AE000584601F0C6FF02E0069801F0C2FF4FEA47
:100AF0006808781CC7B204EBD471B7EB610FECDB6C
:100B0000681CC5B2A542D7DB2DE0002529E00C2CDE
:100B100007D106EB4600284901EB800010F805805C
:100B200004E0264800EB061010F80580002711E0CD
:100B30002048A0F800B008F0010038B10AEB050227
:100B400091B209EB070290B202F018F84FEA680878
:100B5000781CC7B204EBD471B7EB610FE8DB681CFB
:100B6000C5B2A542D3DB13490298088014484088D7
:100B7000401E83B212480088401E82B200210846FF
:100B800001F0C8FF07B0BDE8F08F2DE9FE4306462F
:100B90000F4615461C46DDF8288025E008480088E9
:100BA000401EB04204DB06484088401EB84209DAC5
:100BB000BDE8FE832E00002062470008D64B0008E7
:100BC0006400002020788DE82101FC480388FC485F
:100BD000028839463046FFF74EFF284605EBD071B4
:100BE00006EB61018EB2641C20787E2802DC20783E
:100BF0002028D3DA00BFDBE710B50246012000E071
:100C000050430B00A1F10104E1B2F9D110BD2DE96F
:100C1000FF4F83B0074691461E46109C4FF0000AD6
:100C2000002543E0701B401EC1B20A20FFF7E4FF1D
:100C3000B9FBF0F00A21B0FBF1F201FB1208BAF1A6
:100C4000000F1BD1701EA84218DDB8F1000F13D1A0
:100C500000202021A346CDE90014029004EBDB71B3
:100C6000491001FB057188B2D4490B88D4490A8820
:100C70000499FFF700FF17E04FF0010A002108F187
:100C80003000C0B2A346CDE90141009004EBDB7116
:100C9000491001FB057188B2C8490B88C8490A8808
:100CA0000499FFF7E8FE00BF681CC5B2B542B9DB86
:100CB00007B0BDE8F08F2DE9FC5F054688469146F8
:100CC0009A46DDF830B000954B20019000245FE09B
:100CD00004EB0410BB4911F810009BF80010884287
:100CE00053D104EB0410B74901EB400040789BF866
:100CF0000110884249D108F10F0083B205F10F00BD
:100D000082B24146284601F005FF00263BE000275D
:100D100034E00D9890B904EB0410AA4901EB4000AF
:100D2000801C805D80213941084018B1484601F09F
:100D3000A0FE21E0504601F09CFE1DE0A048A0F876
:100D4000009004EB04109F4901EB4000801C805D83
:100D500080213941084018B14146284601F00EFF74
:100D6000681C85B20098281A102805D1009D08F14A
:100D700001001FFA80F803E0781CC7B2082FC8DB17
:100D800000BF701CC6B2202EC1DB00BF601C84B245
:100D9000019884429CDB8C484088401E83B28A487C
:100DA0000088401E82B20021084601F0B3FEBDE873
:100DB000FC9F2DE9FC5F0546884691469A46DDF882
:100DC00030B0009507200190002467E004EB840018
:100DD00000EB44107D4911F810009BF80010884288
:100DE00059D104EB840000EB4410784901EB40003A
:100DF00040789BF8011088424DD108F1170083B26A
:100E000005F1170082B24146284601F083FE002614
:100E10003FE0002738E00D98A0B904EB840000EB18
:100E200044106A4901EB4000801C805D80213941FB
:100E3000084018B1484601F01CFE23E0504601F07E
:100E400018FE1FE05E48A0F8009004EB840000EB61
:100E500044105E4901EB4000801C805D80213941D7
:100E6000084018B14146284601F088FE681C85B24A
:100E70000098281A182805D1009D08F101001FFAD2
:100E800080F803E0781CC7B2082FC4DB00BF701CD9
:100E9000C6B2482EBDDB00BF601C84B201988442FC
:100EA00094DB49484088401E83B247480088401E72
:100EB00082B20021084601F02DFEBDE8FC9F2DE91D
:100EC000FC5F0546884691469A46DDF830B00095AD
:100ED0000420019000245FE004EB84103C4911F8E9
:100EE00010009BF80010884253D104EB841038495D
:100EF00001EB400040789BF80110884249D108F18D
:100F00001F0083B205F11F0082B24146284601F05E
:100F100001FE00263BE0002734E00D9890B904EB79
:100F200084102B4901EB4000801C805D80213941F9
:100F3000084018B1484601F09CFD21E0504601F000
:100F400098FD1DE01E48A0F8009004EB8410204995
:100F500001EB4000801C805D80213941084018B1C0
:100F60004146284601F00AFE681C85B20098281AFE
:100F7000202805D1009D08F101001FFA80F803E048
:100F8000781CC7B2082FC8DB00BF701CC6B2802E09
:100F9000C1DB00BF601C84B2019884429CDB0A481C
:100FA0004088401E83B208480088401E82B200215B
:100FB000084601F0AFFDBDE8FC9F000030000020B6
:100FC0002E000020C651000864000020BC5B000811
:100FD000C25D00082DE9FF4F83B006468846914662
:100FE000DDE91147109DB2464FF0000B71E0BBF1F7
:100FF000000F40D104EBD4715E4A1288A2EB61016C
:10100000B14204DB5B494988091B414502DA07B05C
:10101000BDE8F08F2878802802DD4FF0010B58E002
:1010200028780D2806D108EB04001FFA80F85646F0
:101030006D1C1EE0102C0DDD102128788DE883003A
:101040004A4641463046069BFFF715FD06F108006B
:1010500086B20EE028788DE891004A464146304637
:10106000069BFFF708FD204604EBD07106EB6101FB
:101070008EB26D1C2DE03F480088001BB04204DB9F
:101080003C484088001B404500DAC0E74FF0000BA9
:10109000202C08D1CDE900574A4641463046069BF0
:1010A000FFF70DFF12E0182C08D1CDE900574A4692
:1010B00041463046069BFFF77CFE07E0CDE900572E
:1010C0004A4641463046069BFFF7F5FDAD1C3019F8
:1010D00086B2287800288AD100BF98E72DE9FE4F14
:1010E0000E4617469846DDE90D9A0C9C204603F003
:1010F00025FA85B21F490988A1EBC50000EBD07124
:10110000C1F34F0B43463A46314658468DE8100628
:10111000FFF760FFBDE8FE8F2DE9F04706460F465A
:10112000154607F1270083B206F1270082B239463F
:10113000304601F0EFFC00240AE015F8149005EBAE
:10114000440090F8018049EA082001F092FC641CF8
:10115000B4F5C86FF1DB07484088401E83B20548EC
:101160000088401E82B20021084601F0D3FCBDE891
:10117000F08700006400002000F09BF8482003F096
:1011800019F801F0C2FD17E000F04FF901F055FA2F
:1011900000F089F900F02CFA00F0EEFA00F025FCDE
:1011A00000F0CCFB00F00FFD00F04AFD01F0D5FA95
:1011B00000F066FE01F037FAE6E7704700BFFEE791
:1011C00000BFFEE700BFFEE700BFFEE770477047C5
:1011D000704770470CB50020019000906C48006883
:1011E00040F480306A49086000BF6948006800F434
:1011F000003000900198401C0190009818B90198A7
:10120000B0F5A06FF1D16248006800F4003010B171
:101210000120009001E0002000900098012843D1B7
:101220005C48006840F010005A49086008460068B1
:1012300020F0030008600846006840F002000860E3
:10124000534840685249486008464068486008462C
:10125000406840F4806048600846406820F47C1094
:1012600048600846406840F4E81048600846006856
:1012700040F08070086000BF4548006800F00070D2
:101280000028F9D04248406820F0030040494860F7
:101290000846406840F00200486000BF3C48406893
:1012A00000F00C000828F9D10CBD10B5FFF792FF33
:1012B00010BD10B53648006840F0010034490860A0
:1012C000084640683449084031494860084600688B
:1012D000324908402E4908600846006820F4802002
:1012E00008600846406820F4FE0048604FF41F0084
:1012F0008860FFF7DAFF4FF000602949086010BDF1
:1013000010B5002100200022214B5B6803F00C0186
:1013100021B1042906D0082928D107E0214B224C0D
:10132000236027E01F4B204C236023E0184B5B68B1
:1013300003F47010164B5B6803F48032022303EB56
:10134000904022B9194B4343174C23600DE0104BDA
:101350005B6803F4003323B1144B4343124C236006
:1013600003E0104B4343104C236003E00D4B0E4C45
:10137000236000BF00BF064B5B68C3F303130C4C34
:10138000E15C094B1B68CB40074C236010BD00009B
:1013900000100240002002400000FFF8FFFFF6FEB0
:1013A00008ED00E000127A000000002000093D0076
:1013B000040000203EB504464FF6FF7001F0F6FB36
:1013C0001F200090FE480288142300210846FEF7E3
:1013D0000BFF1F200090FA48438802884088143889
:1013E00081B20020FEF700FF4FF6FF70F54908803C
:1013F000012010211F234FF6FF72CDE9004102901A
:1014000002210020FFF76AFE01201021EEA2CDE9A3
:1014100000210290EA484088123881B21F234FF61B
:10142000FF720020FFF75AFE3EBD0EB5ECA0FFF79D
:10143000C1FF01201021F0A21F23CDE9002102905D
:10144000DA021E210020FFF749FE01201021E6A24A
:101450001F23CDE900210290DA023C210020FFF792
:101460003DFE01201021E7A21F23CDE900210290BB
:101470004FF61F025A210020FFF730FE01201021F5
:10148000E7A21F23CDE9002102901A46782100200F
:10149000FFF724FE40F2DC5002F0A6FE40F2DC50E2
:1014A00002F0A2FE0EBD0EB54FF6FF700090C448CC
:1014B0004388028800210846FEF796FE012010218D
:1014C000DEA24FF6E073CDE90021029000221E213A
:1014D0001420FFF77FFD4FF4487002F085FE0020D6
:1014E0000090B7484388028800210846FEF77CFE3A
:1014F00001201021D3A24FF6E073CDE90021029024
:101500004FF6FF721E211420FFF764FD4FF4487060
:1015100002F06AFE4FF478400090A94843880288A0
:1015200000210846FEF760FE01201021C7A24FF6F9
:10153000E073CDE9002102901F221E211420FFF745
:1015400049FD4FF4487002F04FFE4FF4FC600090EC
:101550009B484388028800210846FEF745FE01208B
:101560001021BCA24FF6E073CDE9002102901F22AA
:101570001E211420FFF72EFD4FF4487002F034FEB8
:101580001F2000908E484388028800210846FEF7FD
:101590002BFE01201021B1A24FF6E073CDE900210E
:1015A00002904FF478421E211420FFF713FD4FF4F0
:1015B000487002F019FE48F230400090804843889D
:1015C000028800210846FEF70FFE01201021A5A287
:1015D0004FF6E073CDE9002102904FF61F021E2165
:1015E0001420FFF7F7FC4FF4487002F0FDFD0EBD2C
:1015F0002DE9F84300249DA0FFF7DCFE4FF6FF70B5
:1016000000906F484088143883B26D4802881421D6
:101610000020FEF7E9FD00BF48E09A4830F81400CA
:1016200068490880DFF898C1BCF8025005EBD57C0A
:101630004FEA6C0CACF1500CC4EB0419CC440CF127
:101640003C0C1FFA8CF3DFF878C1BCF8006006EBA5
:10165000D67C4FEA6C0CACF1500CC4EB0419CC44B2
:101660000CF13C0C1FFA8CF2DFF854C1BCF802708C
:1016700007EBD77C4FEA6C0CACF1500CC4EB0419AF
:10168000CC441FFA8CF1DFF838C1BCF8008008EBBD
:10169000D87C4FEA6C0CACF1500CC4EB0419CC4470
:1016A0001FFA8CF0FEF713FF601CC4B2052CB4DBEC
:1016B00040F2DC5002F098FD4FF6FF700090404879
:1016C0004088143883B23E48028814210020FEF777
:1016D0008BFD002448E06B4830F81400394908803D
:1016E000DFF8DCC0BCF8026006EBD67C4FEA6C0C7D
:1016F000ACF1500CC4EB0419CC440CF13C0C1FFAB7
:101700008CF3DFF8BCC0BCF8007007EBD77C4FEA65
:101710006C0CACF1500CC4EB0419CC440CF13C0C37
:101720001FFA8CF2DFF898C0BCF8028008EBD87C76
:101730004FEA6C0CACF1500CC4EB0419CC441FFA0A
:101740008CF1DFF87CC0BCF8005005EBD57C4FEA8B
:101750006C0CACF1500CC4EB0419CC441FFA8CF0A7
:10176000FEF7D5FE601CC4B2052CB4DB40F2DC50A1
:1017700002F03AFDBDE8F883F8B5002442A0FFF777
:1017800019FE4FF6FF7000900D484088143883B260
:101790000B48028814210020FEF726FD00BF90E0D0
:1017A0000020074B00905D8805EBD5735B10323B42
:1017B00004EBC40707EB0417D919014B1E886FE02F
:1017C000640000202E000020687474703A2F2F7778
:1017D00077772E6C636477696B692E636F6D000099
:1017E000C8ABB6AFB5E7D7D3D7DBBACFB2E2CAD46E
:1017F000B3CCD0F200000000C8ABB6AFB5E7D7D38A
:1018000000000000322E38222049505320494C4914
:101810003933343120323430583332300000000054
:101820007869616F46656E674051447465636820EE
:10183000323032332D30352D323000005748495484
:1018400045000000424C41434B00000052454420FB
:1018500000000000475245454E200000424C5545CF
:10186000200000004752415900000000B2E2CAD4F3
:10187000333A475549BED8D0CECCEEB3E4B2E2CA33
:10188000D400000014000020B2E2CAD4343A475514
:1018900049BBADD4B2CCEEB3E4B2E2CAD40000008E
:1018A00006EBD6735B10503B04EBC40707EB041741
:1018B000D819FE4B33F814201E23FEF766FD601C7A
:1018C000C4B2052CFFF66CAF40F2DC5002F08CFC89
:1018D0004FF6FF700090F6484088143883B2F44801
:1018E000028814210020FEF77FFC00241FE0012065
:1018F000EF4B00905D8805EBD5735B10323B04EB3A
:10190000C40707EB0417D919E94B1E8806EBD673F9
:101910005B10503B04EBC40707EB0417D819E34BEB
:1019200033F814201E23FEF730FD601CC4B2052CD2
:10193000DDDB40F2DC5002F057FCF8BD0EB5DDA057
:10194000FFF738FD00200C21DFA24FF6E073CDE950
:10195000002102901F221E210A20FFF73BFB0120DD
:101960000C21E4A24FF6E073CDE9002102901F2282
:101970002D210A20FFF72EFB00200C21E8A24FF6B4
:10198000E073CDE9002102901F223C210A20FFF7DD
:1019900021FB00201021EAA24FF6E073CDE90021DF
:1019A00002901F2250210A20FFF714FB0120102172
:1019B000EEA24FF6E073CDE9002102901F226421D0
:1019C0000A20FFF707FB00201021F3A24FF6E07377
:1019D000CDE9002102901F2278210A20FFF7FAFAB0
:1019E0004FF4966002F000FC0EBD2DE9FC5F002470
:1019F000F1A0FFF7DFFC4FF6FF700090AC48408885
:101A0000143883B2AA48028814210020FEF7ECFBA8
:101A100000BF5DE0A54830F81400EE490880A448F6
:101A2000458805EBD57040101438C4EB0411084408
:101A300081B29F48068806EBD6704010153804EB3B
:101A4000840200EB820080B2DFF864C2CDE90001BD
:101A5000BCF8027007EBD77C4FEA6C0CACF1490C78
:101A6000C4EB041BDC441FFA8CF3DFF844C2BCF85F
:101A7000008008EBD87C4FEA6C0CACF1330C04EB23
:101A8000840B0CEB8B0C1FFA8CF2DFF824C2BCF831
:101A9000029009EBD97C4FEA6C0CACF1140CC4EB4E
:101AA000041BDC441FFA8CF1DFF804C2BCF800A070
:101AB0000AEBDA7C4FEA6C0CACF1500C04EB840BB3
:101AC0000CEB8B0C1FFA8CF0FEF7AFFE601CC4B25F
:101AD000052C9FDB40F2DC5002F086FB4FF6FF70D6
:101AE000009073484088143883B2714802881421EA
:101AF0000020FEF779FB00245DE06C4830F814000C
:101B0000B44908806A48458805EBD5704010143800
:101B1000C4EB0411084481B26548068806EBD67010
:101B20004010153804EB840200EB820080B2DFF82D
:101B300080C1CDE90001BCF8027007EBD77C4FEA09
:101B40006C0CACF1490CC4EB041BDC441FFA8CF3A5
:101B5000DFF85CC1BCF8008008EBD87C4FEA6C0C65
:101B6000ACF1330C04EB840B0CEB8B0C1FFA8CF2F6
:101B7000DFF83CC1BCF8029009EBD97C4FEA6C0C51
:101B8000ACF1140CC4EB041BDC441FFA8CF1DFF83D
:101B900020C1BCF800A00AEBDA7C4FEA6C0CACF177
:101BA000500C04EB840B0CEB8B0C1FFA8CF0FEF743
:101BB0005DFE601CC4B2052C9FDB40F2DC5002F0DD
:101BC00013FBBDE8FC9F0EB583A0FFF7F3FB0020DD
:101BD000102186A24FF6E073CDE9002102901F226A
:101BE0001E210A20FFF7F6F90020102188A24FF6E7
:101BF000E073CDE9002102901F2232210A20FFF775
:101C0000E9F90120182188A24FF6E073CDE90021FF
:101C100002901F2246210A20FFF7DCF90120202133
:101C200087A24FF6E073CDE9002102901F226421C4
:101C30000A20FFF7CFF94FF4966002F0D5FA0EBDF7
:101C40000EB583A0FFF7B6FB864A1E210846FFF7B4
:101C500063FA0120102184A24FF6E073CDE9002140
:101C600002901F224B212A20FFF7B4F97D4A1E2142
:101C70005A20FFF751FA012010217BA24FF6E073A2
:101C8000CDE9002102901F224B216620FFF7A2F927
:101C9000744A1E219620FFF73FFA0120102172A2FC
:101CA0004FF6E073CDE900210290DFE01400002040
:101CB00064000020B2E2CAD4363AD3A2CEC4CFD454
:101CC000CABEB2E2CAD40000365831323A61626309
:101CD0006465666768696A6B6C6D6E6F707172734C
:101CE0007475767778797A303132333435363738DF
:101CF00039000000365831323A41424344454647A4
:101D000048494A4B4C4D4E4F5051525354555657DB
:101D100058595A30313233343536373839000000AB
:101D2000365831323A7E21402324255E262A28293E
:101D30005F2B7B7D3A3C3E3F2F7C2D2B2E000000FD
:101D4000385831363A6162636465666768696A6B00
:101D50006C6D6E6F707172737475767778797A3096
:101D6000313233343536373839000000385831369F
:101D70003A4142434445464748494A4B4C4D4E4FF1
:101D8000505152535455565758595A3031323334B2
:101D90003536373839000000385831363A7E214020
:101DA0002324255E262A28295F2B7B7D3A3C3E3F53
:101DB0002F7C2D2B2E000000B2E2CAD4353A4755B5
:101DC0004920547269616E676C65CCEEB3E4B2E28F
:101DD000CAD400002E000020B2E2CAD4373AD6D0CE
:101DE000CEC4CFD4CABEB2E2CAD400003136583114
:101DF000363AC8ABB6AFB5E7D7D3BCBCCAF5D3D07B
:101E0000CFDEB9ABCBBEBBB6D3ADC4FA0000000089
:101E100031365831363A57656C636F6D65C8ABB66D
:101E2000AFB5E7D7D300000032345832343AC9EEA8
:101E3000DBDACAD0D6D0CEC4B2E2CAD400000000E9
:101E400033325833323AD7D6CCE5B2E2CAD40000A6
:101E5000B2E2CAD4383ACDBCC6ACCFD4CABEB2E224
:101E6000CAD40000CC5F0008515100001F224B2152
:101E7000A220FFF7AFF84FF4966002F0B5F90EBD5F
:101E800010B588B00024FE4B0FCBCDE90623CDE979
:101E9000040100BF23E0204600F0EAFEF9A0FFF7AE
:101EA00089FA0121102204A850F824004FF6E073AB
:101EB000CDE9012100901F221E211420FFF78AF88E
:101EC000F54A32211E20FFF727F94FF47A7002F00D
:101ED0008BF94FF47A7002F087F9601CC4B2042CBD
:101EE000D9DB002000F0C4FE08B010BD0EB5EBA099
:101EF000FFF760FA0120EE4900900988203988B286
:101F0000ECA310220221FEF740FE4FF47840EA498C
:101F1000088060E0E94948688047E848007C00F0B4
:101F20000100002853D0E5480089E149098888422A
:101F300051DAE2488089DE49498888424BDABDF8A7
:101F400008004FF6FF71884207D1DC480089ADF8E0
:101F50000800DA488089ADF80A00D8480189D448D9
:101F60000088203881421BDDD4488089122817DA86
:101F70004FF6FF70D14908810881C8A0FFF71AFA0F
:101F80000120CB4900900988203988B2C9A31022CA
:101F90000221FEF7FAFD4FF47840C74908800DE0B2
:101FA0004FF478400221C54CCDE90010A389228965
:101FB000BDF80A10BDF80800FEF734FABF480089E2
:101FC000ADF80800BD488089ADF80A0003E04FF67F
:101FD000FF70ADF808009DE700B587B0B8A0FFF727
:101FE000E9F90020B4490880B1480088069000EB68
:101FF000D0704010323080B20490AD480088059017
:1020000000EBD0704010323880B25523039023216A
:10201000049AFEF75CFA4FF47840A7490880A44878
:102020000088069000EBD0704010401E80B20490F3
:102030009F480088059000EBD0704010313880B286
:10204000542303902421049AFEF761FA1F209A4931
:10205000088097480088069000EBD070401031301F
:1020600080B2049092480088059000EBD070401038
:10207000542303902421049AFEF749FA4FF6FF7087
:102080008D4908800120009089480088069000EB67
:10209000D0704010203880B28EA3102234210590D9
:1020A000FEF773FD48F23040834908800A20009013
:1020B0007F480088069000EBD07040106E3080B2F0
:1020C00004907B480088059000EBD07040106E387B
:1020D00080B2862303907321049AFEF76FFB4FF6BC
:1020E0001F00754908800A200090714800880690FA
:1020F00000EBD07040100A3080B204906C48008829
:10210000059000EBD07040106E3880B286230390AB
:102110007321049AFEF752FB65480088069001205F
:102120000090069800EBD07040100A2340F2CF12C6
:102130007D210590FEF729F94FF478405E4908802B
:10214000102000905A480088069000EBD070401094
:102150000C3880B2032332225F210590FEF757FD31
:1021600000205549088008200090514800880690BA
:1021700000EBD07040101E3080B204904C480088B4
:10218000059000EBD07040101E3880B2D22303902F
:10219000B421049AFEF7C5FA4AF251604649088014
:1021A0000720009042480088069000EBD070401055
:1021B0001D3080B204903E480088059000EBD0703E
:1021C00040101D3880B2D0230390B521049AFEF749
:1021D000F5FA4FF61F003849088001200090344876
:1021E0000088069000EBD07040100F3880B23AA300
:1021F0001022BB210590FEF7C8FC0120102138A257
:10220000CDE9002102902A480088069000EBD070AA
:1022100040102F3880B24FF6FF734FF478429B2165
:102220000590FEF7D7FEFAE1244840680690804703
:102230002248007C00F001000028F4D01F4880896B
:1022400023287DDD1D488089552879DA18480088C3
:10225000059000EBD0704010323818490989884247
:102260006FDA13480088069000EBD0704010401ED3
:1022700012490989884264DD4FF478400E4937E0FD
:10228000506C0008B2E2CAD431303AC6C1C4BBD0E7
:10229000FDD7AAB2E2CAD400CC5F0008B2E2CAD429
:1022A00031323AB4A5C3FE50454EB2E2CAD4000062
:1022B00064000020525354002E00002034000020FF
:1022C000B2E2CAD431313AB4A5C3FEB0B4BCFCB258
:1022D000E2CAD4004F4E00004558495400000000A7
:1022E000B0B445584954BCFCCDCBB3F60000000057
:1022F0000880F8480088069000EBD0704010401E1F
:1023000080B20490F3480088059000EBD070401034
:10231000313880B2542303902421049AFEF7F7F851
:102320001F20ED490880EB480088069000EBD07034
:102330004010313080B20490E6480088059001E0FA
:102340007AE01DE000EBD07040105423039024216C
:10235000049AFEF7DCF84FF6FF70DF490880012091
:102360000090DC480088069000EBD07040102038C8
:1023700080B2AFF2A003102234210590FEF705FCD5
:10238000D4480088059000EBD0704010D3490989EB
:10239000884251DACF480088069000EBD070401098
:1023A0003230CE490989884246DD1F20CA4908805B
:1023B000C8480088069000EBD0704010401E80B2E4
:1023C0000490C4480088059000EBD070401031386C
:1023D00080B2542303902421049AFEF798F84FF416
:1023E0007840BD490880BB480088069000EBD0705B
:1023F0004010313080B20490B6480088059000EB60
:10240000D0704010542303902421049AFEF77FF8E3
:102410004FF6FF70B049088001200090AD48008859
:10242000069000EBD07040100D3080B2ACA31022AB
:1024300034210590FEF7A9FBA6480088059000EB23
:10244000D07040106438A5490989884275DCA148DC
:102450000088069000EBD070401064309F490989D5
:1024600088426ADB9D488089732866DD9B488089A5
:10247000862862DA48F23040974908800A200090A6
:1024800094480088069000EBD07040106E3080B207
:102490000590924800890A3880B2862304907321FF
:1024A000059AFEF78BF94FF61F008B4908800A202A
:1024B000009088480088069000EBD07040106E387D
:1024C00080B20490854800890A3080B28623024693
:1024D000732105900498FEF771F9012000907F4860
:1024E00000890A2340F2CF127D210690FDF74DFFAF
:1024F0004FF478407849088076480088059000EBD2
:10250000D0704010643875490989081A0690102067
:10251000009070480088049000EBD07040100C3898
:1025200080B20290069800EBD07040100323024660
:102530005F2103900298FEF76AFB664800880590C9
:1025400000EBD07040101E3864490989884266DC6F
:1025500060480088069000EBD07040101E305F4944
:10256000098988425BDB5D488089B42857DD5B4878
:102570008089D22853DA4FF6FF7057490880082027
:10258000009054480088069000EBD07040101E3038
:1025900080B204904F480088059000EBD070401046
:1025A0001E3880B2D2230390B421049AFEF7B9F802
:1025B00042F61230484908800720009045480088BC
:1025C000069000EBD07040101D3080B2049041485E
:1025D0000088059000EBD07040101D3880B2D023E9
:1025E0000390B521049AFEF7E9F848F21F403A49F2
:1025F00008800120009037480088069000EBD070DA
:1026000040100F3880B2AFF230331022BB2105905A
:10261000FEF7BBFA4FF6FF703049088100E003E691
:1026200000BF07B000BD10B52C490868804700B155
:1026300010BDFFF7D1FCFFF759FC70B590B000203A
:102640000D900E900F90242104A801F096FF25A074
:10265000FEF7B0FE00F075FC0646324627A10DA835
:1026600001F0FEFD012010210DAA4FF6E073CDE927
:10267000002102901F2219213220FEF7ABFC00241A
:1026800063E0204830F814001349088004EBC400CC
:1026900000EB041000F1410304EBC40000EB041054
:1026A0002D3081B21E220A20FDF731FF04EBC40059
:1026B00000EB041000F13701142000F06BFA05461E
:1026C00005480088A84221D10FA10DA801F012FFF2
:1026D00020E00000640000202E00002034000020D4
:1026E0004F464600B2E2CAD4323AB6C14944BACDE6
:1026F000D1D5C9ABD6B5B2E2CAD4000049443A300C
:10270000782578001E0000204F4B000072A10DA814
:1027100001F0F0FE0DAB2A4671A104A801F0A0FD66
:102720000120102104AACDE90021029004EBC4008D
:1027300000EB04102F3081B24FF6E0736E48028830
:102740002820FEF747FC601CC4B2072C99DB40F23E
:10275000DC5001F049FD10B070BD38B567A0FEF740
:1027600029FE1F2064490880694801F0A5FE012068
:1027700068A31022322100900F20FEF706FA0120F4
:102780006AA31022462100900F20FEF7FEF90120D7
:102790006CA310225A2100900F20FEF7F6F90120B9
:1027A0006EA310226E2100900F20FEF7EEF901209B
:1027B00070A31022822100900F20FEF7E6F901207D
:1027C00072A31022962100900F20FEF7DEF901205F
:1027D00073A31022AA2100900F20FEF7D6F94FF420
:1027E000784045490880002473E0FDF7D7FC42F2A9
:1027F000107190FBF1F201FB1205102005232A460F
:10280000322100906420FEF702FAFDF7C7FC42F285
:10281000107190FBF1F201FB1205102005232A46EE
:10282000462100906420FEF7F2F9FDF7B7FC42F272
:10283000107190FBF1F201FB1205102005232A46CE
:102840005A2100906420FEF7E2F9FDF7A7FC42F25E
:10285000107190FBF1F201FB1205102005232A46AE
:102860006E2100906420FEF7D2F9FDF797FC42F24A
:10287000107190FBF1F201FB1205102005232A468E
:10288000822100906420FEF7C2F9FDF787FC322117
:1028900090FBF1F201FB1205102005232A46962138
:1028A00000906420FEF7B3F9FDF778FC642190FBFB
:1028B000F1F201FB1205102005232A46AA210090FF
:1028C0006420FEF7A4F94FF4FA7001F08DFC601C4F
:1028D000C4B20F2C89DB38BD4552524F5200000064
:1028E0007265616420636F6C6F723A3078253034A2
:1028F00058202025730000002E000020B2E2CAD428
:10290000393AB6AFCCACCAFDD7D6CFD4CABE0000D8
:1029100040E20100204843484F3A20202020202058
:10292000202020202075672F6D3300002020434F8A
:10293000323A202020202020202020202070706D7E
:10294000000000002054564F433A20202020202031
:10295000202020202075672F6D330000504D322E2F
:10296000353A202020202020202020202075672F8D
:102970006D33000020504D31303A2020202020209F
:10298000202020202075672F6D3300002020544523
:10299000503A20202020202020202020204300000A
:1029A000202048554D3A2020202020202020202083
:1029B0002025000010B504464FF40070FE49086061
:1029C000802008602146FD4800F0FCFA4FF40070BA
:1029D000F949091F086010BD10B504464FF4007096
:1029E000F54908608020091F08602146F34800F07F
:1029F000E9FA4FF40070F049091F086010BD10B5E6
:102A00004FF40070EC4908608020091F0860002125
:102A1000EA4800F0E8FAFF21E84800F0D3FA04465B
:102A20000121E64800F0DFFA4FF40070E249091F87
:102A30000860204610BD70B505460C462846FFF7D5
:102A4000B9FFE0B2FFF7C8FF70BD10B504462046DD
:102A5000FFF7B0FFFFF7D3FF10BD10B5D849087AD4
:102A6000FFF7A8FF10BD10B5D549887AFFF7A2FF80
:102A700010BD10B504464FF40070CF4908608020A7
:102A8000091F08602112CD4800F09CFAE1B2CB4842
:102A900000F098FA4FF40070C749091F086010BD94
:102AA00010B5034603F0F800000201F0FC0440EA10
:102AB000C40040EAD20010BD70B58020BE49091F95
:102AC00008608000091D08600021BC4800F08BFAF6
:102AD000FF21BA4800F076FAFF21B84800F072FAF8
:102AE0000446FF21B54800F06DFA0546FF21B348C2
:102AF00000F068FA06460121B04800F074FA4FF47D
:102B00000070AD49091F0860324629462046FFF78C
:102B1000C7FF70BD2DE9F04104460D4616461F461D
:102B2000A749087BFFF746FF2012FFF755FFE0B2E9
:102B3000FFF752FF3012FFF74FFFF0B2FFF74CFFE5
:102B40009F49887BFFF736FF2812FFF745FFE8B261
:102B5000FFF742FF3812FFF73FFFF8B2FFF73CFFE5
:102B6000FFF77BFFBDE8F08170B504460D462B46AC
:102B7000224629462046FFF7CDFF70BD70B50446BA
:102B80000D4629462046FFF7EFFF8E480088FFF7E5
:102B900070FF70BD70B504460D4629462046FFF70C
:102BA000E3FFFFF760FFFFF787FF70BD70B50446D6
:102BB00083484088401E83B281480088401E82B20C
:102BC00000210846FFF7A6FF4FF400707A4908601D
:102BD0008020091F086000250FE0002608E0211270
:102BE000764800F0EFF9E1B2744800F0EBF9761C9A
:102BF00073480088B042F2D86D1C71484088A842E2
:102C0000EBD84FF400706C49091F086070BD08B51F
:102C10000121082001F0E4F84FF47070ADF80000D5
:102C200003208DF8020010208DF8030069466248E9
:102C3000143800F019FE01206349086008BD10B582
:102C40004FF480705C49091F0860322001F0CCFA13
:102C50004FF4807058490860642001F0C5FA4FF4C1
:102C600080705549091F0860322001F0BDFA10BD7F
:102C700010B504462A20524988812B20C8812C2077
:102C800008812E2048812046E11704EB91718910BC
:102C9000A4EB81014A4A91711046807930B1012834
:102CA0000FD0022818D003282CD120E0F02044496E
:102CB00008804FF4A070488008213620FFF7BBFE43
:102CC00021E04FF4A0703E490880F0204880682140
:102CD0003620FFF7B0FE16E0F020394908804FF4A7
:102CE000A0704880C8213620FFF7A5FE0BE04FF406
:102CF000A07033490880F0204880A8213620FFF7D3
:102D00009AFE00E000BF00BF10BD10B500F07EF9D4
:102D1000FFF77DFFFFF793FFCF20FFF74BFE00206B
:102D2000FFF75AFEC120FFF757FE3020FFF754FE91
:102D3000ED20FFF73FFE6420FFF74EFE0320FFF774
:102D40004BFE1220FFF748FE8120FFF745FEE820EA
:102D5000FFF730FE8520FFF73FFE0020FFF73CFE27
:102D60007820FFF739FECB20FFF724FE3920FFF74C
:102D700033FE2C20FFF730FE0020FFF72DFE34201D
:102D8000FFF72AFE0220FFF727FEF720FFF712FECB
:102D90002020FFF721FEEA20FFF70CFE0020FFF7BE
:102DA0001BFE0020FFF718FEC020FFF703FE1320D4
:102DB000FFF712FEC12009E0140C01400030014071
:102DC000640000202E00002098812142FFF7F2FDD0
:102DD0001320FFF701FEC520FFF7ECFD2220FFF7CF
:102DE000FBFD3520FFF7F8FDC720FFF7E3FDBD2011
:102DF000FFF7F2FD2120FFF7DDFD3620FFF7DAFDBA
:102E00000820FFF7E9FDB620FFF7D4FD0A20FFF701
:102E1000E3FDA220FFF7E0FD3A20FFF7CBFD5520B0
:102E2000FFF7DAFDF620FFF7C5FD0120FFF7D4FD1F
:102E30003020FFF7D1FDB120FFF7BCFD0020FFF7E8
:102E4000CBFD1B20FFF7C8FDF220FFF7B3FD0020EC
:102E5000FFF7C2FD2620FFF7ADFD0120FFF7BCFD07
:102E6000E020FFF7A7FD0F20FFF7B6FD3520FFF7A5
:102E7000B3FD3120FFF7B0FD0B20FFF7ADFD0E20B5
:102E8000FFF7AAFD0620FFF7A7FD4920FFF7A4FDE5
:102E9000A720FFF7A1FD3320FFF79EFD0720FFF7D6
:102EA0009BFD0F20FFF798FD0320FFF795FD0C20F9
:102EB000FFF792FD0A20FFF78FFD0020FFF78CFD42
:102EC000E120FFF777FD0020FFF786FD0A20FFF7DE
:102ED00083FD0F20FFF780FD0420FFF77DFD11200B
:102EE000FFF77AFD0820FFF777FD3620FFF774FD26
:102EF0005820FFF771FD4D20FFF76EFD0720FFF70B
:102F00006BFD1020FFF768FD0C20FFF765FD3220F8
:102F1000FFF762FD3420FFF75FFD0F20FFF75CFD38
:102F20001120FFF747FD782001F05EF92920FFF717
:102F300041FD0020FFF79CFE4FF6FF70FFF736FEC5
:102F400010BD38B500200090012411E0D920FFF712
:102F500031FD04F11001C8B2FFF73EFDD320FFF7A9
:102F600029FDFFF74CFD611E0DF80100601CC4B285
:102F7000042CEBDB9DF80100094988800846808815
:102F80004FF6FF7101EA00200549888008468088D5
:102F90009DF802100843024988800846808838BDA1
:102FA0006400002010B500F00EFA08B1012010BD39
:102FB0000248034948600020F9E700009734000800
:102FC00034000020024600BF108900F002000028F3
:102FD000FAD0918100BF108900F001000028FAD0DA
:102FE0009089C0B2704702884FF6C7731A400280BA
:102FF000012902D10288028003E0028842F0100217
:103000000280028842F040020280704700B587B01B
:103010000121052000F0E4FEA020ADF8040003200B
:103020008DF8060018208DF8070001A91C4800F053
:103030001BFC4020ADF8040048208DF80700032059
:103040008DF8060001A9164800F00EFC01210803C6
:1030500000F0C6FE0020ADF808004FF48270ADF815
:103060000A000020ADF80C000220ADF80E0001208F
:10307000ADF810004002ADF812000020ADF81400C9
:10308000ADF816000720ADF8180002A9054800F0B9
:1030900031FF0121034800F0D2FF07B000BD00005E
:1030A000000801400030014010B5012001F0B8F8DF
:1030B00010BD08B501210C2000F092FE4FF4007005
:1030C000ADF8000010208DF8030003208DF80200F9
:1030D00069468C4800F0C8FB2020ADF80000694626
:1030E000894800F0C1FB0120884908608849C1F87F
:1030F000A40108BD10B58348001D006820F0F00051
:103100008049091D08600846006840F030000860EA
:103110000120804908608049C1F89401FFF7C4FF8D
:1031200000207C490860FFF7BFFF00207A49C1F802
:10313000940110BD10B57348001D006820F0F00028
:103140007049091D08600846006840F030000860BA
:1031500000206E4908606E49C1F8A401FFF7A4FF82
:1031600001206A490860FFF79FFF01206849C1F804
:10317000A40110BD10B500246248001D006820F0B5
:10318000F0006049091D08600846006840F08000B2
:10319000086001205F49086001F042F801205E49A3
:1031A000C1F8940101F03CF807E0601CC4B2FA2CAD
:1031B00003DDFFF7BFFF012010BD564880380068CF
:1031C0000028F2D15149086000BFF5E710B5002092
:1031D0004E4908604B48001D006820F0F000494946
:1031E000091D08600846006840F0300008600020B3
:1031F0004749C1F8A401FFF757FF01204349086080
:10320000FFF752FF00204449C1F8940110BD10B5EA
:1032100000203E4908603B48001D006820F0F00097
:103220003849091D08600846006840F03000086011
:1032300001203749C1F8A401FFF736FF01203349C7
:103240000860FFF731FF00203349C1F8940110BD39
:1032500070B504462B48001D006820F0F000294995
:10326000091D08600846006840F030000860002032
:1032700026490860002511E0E0092649086060063B
:10328000040E01202449C1F89401FFF70DFF00202E
:103290001E490860FFF708FF681CC5B2082DEBDB6C
:1032A00070BD70B5054600241648001D006820F06A
:1032B000F0001449091D08600846006840F08000CD
:1032C0000860002613E0002010490860032000F089
:1032D000A7FF01201049C1F894016006040E0D48B3
:1032E0008038006808B1601CC4B2701CC6B2082ED9
:1032F000E9DB15B9FFF78BFF01E0FFF767FF204619
:1033000070BD000000080140000C01409481214282
:1033100000002142A4012142008021422DE9F04118
:1033200005460E4617464FF00008FFF7E3FE7020F3
:10333000FFF78EFFFFF71EFFE8B2FFF789FFFFF7E9
:1033400019FF00240BE0305DFFF782FFFFF712FF4B
:103350008046B8F1000F00D003E0601CC4B2BC424C
:10336000F1DB00BFFFF7E6FE4046BDE8F0812DE946
:10337000F04106460F461546FFF7BCFE7020FFF7EA
:1033800067FFFFF7F7FEF0B2FFF762FFFFF7F2FE0D
:10339000FFF7B0FE7120FFF75BFFFFF7EBFE0024A5
:1033A0000BE0691EA14201D0012100E00021084686
:1033B000FFF777FF3855601CC4B2AC42F1DBFFF772
:1033C000B9FEBDE8F0811CB50121042000F008FD24
:1033D0004FF48060ADF8000010208DF8030003204A
:1033E0008DF802006946A54800F03EFA4FF480616E
:1033F000A24800F0E6FA4FF48070ADF800004820D3
:103400008DF8030069469D4800F02EFA4FF4807154
:103410009A4800F0D6FAFFF74CFE00209849086061
:103420000A2000F0E1FE01209649C1F8A8014FF4FE
:10343000FA7000F0D9FE012201A9A820FFF797FF3A
:103440009DF80400112801D001201CBD022201A911
:103450009F20FFF78CFF9DF80400262801D0012053
:10346000F3E79DF8050048B19DF80500012805D057
:103470009DF80500022801D00120E6E7012201A9FC
:10348000A320FFF774FF9DF80400642801D00120F9
:10349000DBE70020D9E77CB5002400267A480078D5
:1034A000401C79490870084600780A2190FBF1F227
:1034B00001FB120018B1744800780A287EDA012254
:1034C00069460220FFF753FF9DF80000002875D0E1
:1034D0009DF800000328F1DA9DF80010FF208840D5
:1034E000C5B2E843C0B240F0C00068490874002487
:1034F00092E0674931F81400042201A9FFF737FF71
:103500006248007C0121A140084000287DD061482C
:10351000807930B101281DD0022838D0032878D115
:1035200058E09DF805009DF8041001F00F0100EB34
:1035300001205649083121F814009DF807009DF834
:10354000061001F00F0100EB012150480C3020F86B
:1035500014105EE09DF805009DF8041001F00F01C5
:1035600000EB01204B494988081A81B247480C30CA
:1035700020F814109DF807009DF8061001F00F01C7
:1035800000EB01204149083121F8140041E09DF889
:1035900005009DF8041001F00F0100EB01203D49EA
:1035A0000988081A81B23948083020F814109DF8AB
:1035B00007009DF8061001F00F0100E03BE000EB72
:1035C000012034494988081A81B230480C3020F86B
:1035D00014101EE09DF805009DF8041001F00F0185
:1035E00000EB012029490C3121F814009DF8070057
:1035F0009DF8061001F00F0100EB01202549098814
:10360000081A81B22148083000E003E020F81410C5
:1036100000BF00BF601CC4B2022CFFF66AAF0126D7
:103620001A48008920B91948808908B900200090FB
:103630000020154908709DF80000A8B91348007CC7
:1036400000F0800030B11148007C20F080000F496C
:10365000087409E04FF6FF700C490881888108461C
:10366000007C00F0E000087407480078F02802DDD4
:103670000A200549087030467CBD00000008014062
:10368000A80121420000214248000020340000200F
:10369000606C00086400002008480047FEE7FEE771
:1036A000FEE7FEE7FEE7FEE7FEE7FEE7FEE7FEE7F2
:1036B00003480449024A044B70470000ED0000082B
:1036C000B8010020B8030020B801002031490143AF
:1036D000314A1160704770B5002100230F22C47871
:1036E00004B32D4C246804F4E064C4F5E064210ABA
:1036F000C1F10403CA40447804FA03F18478144009
:1037000021430901254C0678A155047804F01F05D2
:103710000124AC4005786D11AD0005F1E025C5F838
:10372000004109E0047804F01F050124AC401C4D61
:103730000678761145F8264070BD1A4A0A400243C1
:10374000154B1B1F1A60704739B1134A121D1268BE
:103750000243114B1B1D1A6006E00F4A121D12682E
:1037600082430D4B1B1D1A607047042808D14FF08F
:10377000E021096941F004014FF0E022116107E006
:103780004FF0E021096921F004014FF0E0221161BE
:10379000704700000000FA050CED00E000E400E0D6
:1037A00080E100E080FFFF1F10B50446CC48844252
:1037B00008D10121042000F02DFB0021042000F09D
:1037C00029FB46E0C748844208D10121082000F0C7
:1037D00021FB0021082000F01DFB3AE0C248844292
:1037E00008D10121102000F015FB0021102000F06D
:1037F00011FB2EE0BD48844208D10121202000F0B9
:1038000009FB0021202000F005FB22E0B84884429B
:1038100008D10121402000F0FDFA0021402000F0F5
:10382000F9FA16E0B348844208D10121802000F063
:10383000F1FA0021802000F0EDFA0AE0AE4884425F
:1038400007D10121801500F0E5FA0021A01500F054
:10385000E1FA10BD10B50121084600F0DBFA0021A5
:10386000012000F0D7FA10BD2DE9F04102460025F5
:103870000026002000230024002791F803C00CF04C
:103880000F0591F803C00CF0100CBCF1000F03D031
:1038900091F802C04CEA050591F800C0BCF1000F98
:1038A00031D0146800202BE04FF0010C0CFA00F32B
:1038B000B1F800C00CEA03069E4220D183004FF00D
:1038C0000F0C0CFA03F7BC4305FA03FC4CEA0404A2
:1038D00091F803C0BCF1280F06D14FF0010C0CFA8F
:1038E00000FCC2F814C00AE091F803C0BCF1480F14
:1038F00005D14FF0010C0CFA00FCC2F810C0401CBE
:103900000828D1D31460B1F800C0BCF1FF0F34DD3A
:10391000546800202EE000F1080C4FF0010808FA6E
:103920000CF3B1F800C00CEA03069E4221D18300DB
:103930004FF00F0C0CFA03F7BC4305FA03FC4CEAFA
:10394000040491F803C0BCF1280F05D100F1080C64
:1039500008FA0CF8C2F8148091F803C0BCF1480FC3
:1039600007D100F1080C4FF0010808FA0CF8C2F872
:103970001080401C0828CED35460BDE8F0814FF67B
:10398000FF710180022181700421C17070470246DD
:10399000002093680B400BB1012000E0002070472D
:1039A0000146886880B2704702460020D3680B4009
:1039B0000BB1012000E0002070470146C86880B2CA
:1039C000704701617047416170470AB1016100E0D1
:1039D00041617047C16070474FF480320A43826191
:1039E0008161826182698269704702460020434B8F
:1039F00018684FF68073184040EA021008433F4BA6
:103A0000186070473E49C8617047F0B50A46002308
:103A100000240021002500F00046B6F1004F02D13D
:103A2000364EF16901E0354E7168C0F3034583B24B
:103A300000F44016B6F5401F08D121F070612F4EFA
:103A4000766826F070662D4F7E6012E000F48016D6
:103A5000B6F5801F06D1032606FA05F4A14341F00E
:103A6000706106E0460D360103FA06F6B14341F0F7
:103A7000706122B1460D360103FA06F6314300F0BB
:103A80000046B6F1004F02D11C4EF16101E01B4E21
:103A90007160F0BD30B500228B071C0F0F2303FAB5
:103AA00004F2164B08338C1053F824309343134C14
:103AB00008348D1044F8253023468C1053F82430F8
:103AC0008C07240F00FA04F423430C4C08348D10A7
:103AD00044F8253030BD0A49DC31086070470000E9
:103AE00000080140000C014000100140001401409A
:103AF00000180140001C014000200140000001406E
:103B000000002042DF48006840F00100DD49086005
:103B100008464068DC490840DA49486008460068C1
:103B2000DA490840D74908600846006820F4802038
:103B300008600846406820F4FE0048604FF41F000B
:103B400088607047CF49096821F48031CD4A1160FF
:103B50001146096821F480211160B0F5803F03D03F
:103B6000B0F5802F0ED106E0C649096841F48031D6
:103B7000C44A116007E0C349096841F4A021C14A61
:103B8000116000E000BF00BF704710B50146002281
:103B9000002300204A11012A02D1BA4C236806E012
:103BA000022A02D1B74C236A01E0B64C636A01F0E5
:103BB0001F02012494401C400CB1012000E00020B1
:103BC00010BD38B5002000900024002500BF312032
:103BD000FFF7DBFF05460098401C00900098B0F509
:103BE000A06F01D0002DF2D03120FFF7CEFF08B139
:103BF000012400E00024204638BD01460020A14AEF
:103C0000106820F0F80040EAC10010607047A04939
:103C100008607047024600209A4B586820F47C10D8
:103C200042EA01031843974B586070479849086669
:103C3000704701460020934A506820F00300084373
:103C4000506070478F48406800F00C007047014694
:103C500000208C4A506820F0F00008435060704704
:103C600001460020874A506820F4E0600843506015
:103C7000704701460020834A506820F4605040EAB3
:103C8000C1005060704729B17E4A527A02437D4B91
:103C90005A7204E07B4A527A82437A4B5A727047D6
:103CA0007B49D8310860704701460020754A50684A
:103CB00020F440400843506070470021714A203290
:103CC0001170704A82F82010012802D004280AD10D
:103CD00004E001216B4A2032117005E00521694A98
:103CE0002032117000E000BF00BF704769490860D2
:103CF00070476449096A0143624A11627047654925
:103D000044390860704730B50021002200240023A8
:103D10005C4D6D6805F00C0121B1042905D008291E
:103D200023D105E05C4D056022E05B4D05601FE09E
:103D3000544D6D6805F47012524D6D6805F4803471
:103D4000022505EB92421CB9544D554305600BE02A
:103D50004C4D6D6805F400351DB1504D554305605F
:103D600002E04D4D5543056002E04B4D056000BF3C
:103D700000BF444D6D6805F0F0010909484D6B5CCA
:103D80000568DD4045603F4D6D6805F4E061090A56
:103D9000434D6B5C4568DD4085603A4D6D6805F4C8
:103DA0006051C90A3E4D6B5C4568DD40C560354DCC
:103DB0006D6805F44041890B3A4D6B5CC568B5FBF5
:103DC000F3F5056130BD29B12E4A526902432D4BEE
:103DD0005A6104E02B4A526982432A4B5A61704768
:103DE00029B1284A92690243264B9A6104E0254A88
:103DF00092698243234B9A61704729B1214AD26963
:103E00000243204BDA6104E01E4AD26982431D4B13
:103E1000DA61704729B11B4AD2680243194BDA6054
:103E200004E0184AD2688243164BDA60704729B121
:103E3000144A12690243134B1A6104E0114A1269D1
:103E40008243104B1A61704712494039086070472D
:103E50000F49C86470470B49C87170470948406AE8
:103E600040F0807007494862704701460020054ACB
:103E700092680A400AB1012000E000207047014921
:103E800088727047001002400000FFF8FFFFF6FE46
:103E9000000042428004424200127A0000093D00C4
:103EA000490000205900002010B50446BE48844255
:103EB00008D101218014FFF7ADFF0021A014FFF706
:103EC000A9FF16E0B948844208D101210014FFF788
:103ED000AEFF00212014FFF7AAFF0AE0B448844295
:103EE00007D10121C013FFF7A2FF0021E013FFF764
:103EF0009EFF10BD10B50022028802F441520B88CB
:103F00004C8823438C882343CC8823430C89234348
:103F10004C8923438C892343CC8923431A43028051
:103F2000838B4FF2FF74234083830B8A038210BD7F
:103F30002DE9F04F85B005460C464FF000090227E9
:103F40004FF000084FF0010B0026B246A88B4FF24D
:103F500040010840A88302202884B5F81C90A0687E
:103F6000022801D100BF38E0A08810B94FF0010B42
:103F700001E04FF0020B8D48854200D100E000BF08
:103F80006846FFF7C0FEDDF800A0E088B0F5007FCE
:103F90000AD14FEA1A2000EB80004000A168B0FB74
:103FA000F1F0401D86B20BE04FEA4B10BAFBF0F087
:103FB00000EB80004000A168B0FBF1F0401D86B22C
:103FC0000A20B6FBF0F606F00108A6EB0800C0F3E5
:103FD0004F074FF6FF7000EA0828022F01DBFF2F82
:103FE00002DD02274FF00008E08840EA080038436D
:103FF0002884A088A1890843618808432188084350
:1040000040F4006040EA0909A5F81C9005B0BDE83D
:10401000F08F0021018041808180C1800181418138
:104020008181C18107210182704700210180418087
:104030008180C1800221816000218181704721B18E
:10404000028842F04002028004E002884FF6BF730B
:104050001A400280704721B1828B42F480628283D1
:1040600004E0828B4FF6FF331A408283704730B5ED
:10407000002400230C110125A540ABB21AB185889C
:104080001D43858002E085889D43858030BD1AB13F
:1040900083880B43838002E083888B43838070474F
:1040A000818170470146888970474FF6FF629142CF
:1040B00004D0028842F48072028004E002884FF645
:1040C000FF631A400280704721B1828842F00402E7
:1040D000828004E082884FF6FB731A40828070472A
:1040E00002884FF2FF731A40028002880A4302805E
:1040F0007047018841F480510180704721B10288E6
:1041000042F40052028004E002884DF6FF731A4028
:104110000280704702460020012901D0108B00E088
:10412000908A70470146088A7047B1F5804F04D1E4
:10413000028842F48042028004E002884BF6FF735A
:104140001A40028070470246002013890B400BB1D1
:10415000012000E000207047CA4302817047F0B59B
:104160000246002000240023002501F00F0701264D
:10417000BE40B4B20B1101269E40B3B2968806EA47
:1041800003051689264016B10DB1012000E000207C
:10419000F0BD10B5002201F00F040123A3409AB234
:1041A000D343038110BD00000030014000380040BF
:1041B000003C004010B504466FF00400FFF7D5FA4C
:1041C000E11704EB5171C1F3C701234A1170104686
:1041D000007800EB4001C1EBC0104FF6FF7101EA1F
:1041E000C0001E49088010BD01461C4A12884A437F
:1041F0004FF0E0235A6100229A6101221A6100BF48
:104200004FF0E022106900F001021AB100F4803290
:10421000002AF5D000224FF0E0231A619A6170471E
:1042200001460D4A12784A434FF0E0235A610022BA
:104230009A6101221A6100BF4FF0E022106900F07C
:1042400001021AB100F48032002AF5D000224FF0AA
:10425000E0231A619A6170475E0000206000002030
:104260000FB41CB5074B06AA7B446946009005981D
:1042700000F00BFA0020694600F01AFA1CBC5DF849
:1042800014FB00004504000070B504468569006811
:10429000C10601D5302600E02026C00707D070BD3A
:1042A000D4E9012130469047206A401C20626D1EEF
:1042B000F6D570BD70B5044685690078C00707D192
:1042C00070BDD4E9012120209047206A401C206263
:1042D0006D1EF6D570BD70B50C460546012A05D099
:1042E0002878800600D5EA69002302E0012305E072
:1042F0005B1C934202D2E05C0028F9D1A869E61861
:10430000C01AA861286A184428622846FFF7BCFF33
:1043100004E0D5E9012114F8010B9047B442F8D329
:104320002846FFF7C7FF70BD70B504460D4621460D
:104330001068AFF300802188090502D50F4A7A443E
:1043400002E00E4A7A440E32002104F1240305E013
:1043500000F00F060009965D5E54491C0028F7D155
:1043600020780023000704D5702D02D009B1022364
:1043700011322046BDE8704000F029B92229000022
:104380002DE9F05F894604464FF0000ADFF824B1BA
:10439000FB44C0F820A02046E168884700287DD073
:1043A000252806D0D4E901219047206A401C2062CC
:1043B000F1E700255F462046E16888472028064649
:1043C00007DB312E05D2B81910F8200C08B10543CF
:1043D000F1E7A80701D525F00405C4F81CA00027C3
:1043E000C4F818A02A2E09D0304600F0B3F938B32B
:1043F00004EB8708303EC8F8186019E059F8041B30
:10440000204604EB87029161E1688847012F064648
:1044100018D1E069002820DA25F020051DE0D8F841
:10442000180000EB800006EB40003038C8F8180098
:104430002046E1688847064600F08CF90028EED156
:10444000012F0AD02E2E08D12046E16888477F1C14
:104450000646022F45F02005C4DBA069002803DAD8
:10446000404245F00105A061E80701D025F01005A4
:10447000A6B1A6F14100192802D8203645F40065FE
:104480004A463146204625604D46FBF769FE60B13D
:10449000012807D0ED1D25F0070000E007E000F13E
:1044A000080978E705F1040975E730467AE7206ADC
:1044B000BDE8F09FF82800000B4910B5A1F17C027F
:1044C0000A4CC2E93712372106E000EB104342F8EC
:1044D0002130074B00FB03400B1EA1F10101F4DC6E
:1044E00010BD0120E8E70000F0000020E119D666C9
:1044F000CD0D010040EA0103024630B59B0710D103
:104500004FF0013400E008C208C91D1B9D4315EAA5
:10451000C41FF8D013F0FF0102F8011B0DD01B0AD5
:10452000F8E711F8013B002B02F8013B05D011F828
:10453000013B002B02F8013BF3D130BD10B5431C09
:1045400002E010F8011B71B18107FAD14FF001327E
:1045500002C88C1A8C4314EAC211F9D0C01A0A0698
:1045600003D0C01E10BDC01A10BD0A0401D0801EA9
:1045700010BD0902FCD0401E10BD4FF0000200B576
:10458000134694469646203922BFA0E80C50A0E876
:104590000C50B1F12001BFF4F7AF090728BFA0E824
:1045A0000C5048BF0CC05DF804EB890028BF40F8F0
:1045B000042B08BF704748BF20F8022B11F0804F32
:1045C00018BF00F8012B70477047704770472DE9FE
:1045D000F0470D4699469246044600F124080168CA
:1045E000880604D5E06921F01001216000E0012077
:1045F000A84201DD471B00E00027A1697A1902EB00
:104600000900081AA0612078C00602D42046FFF7EE
:104610003BFE002608E0D4E901211AF80600904785
:10462000206A401C761C20624E45F4DB2078C006D0
:104630000AD52046FFF728FE06E0D4E90121302004
:104640009047206A401C2062381EA7F10107F4DC65
:1046500007E0D4E9012118F805009047206A401CC2
:104660002062281EA5F10105F3DC2046FFF722FE9B
:104670002078000602D50220BDE8F0870120FBE784
:1046800001694A1C02610878704700B58FB0CDE916
:1046900001310021059105497944CDE90310114606
:1046A0006846FFF76DFE0FB000BD0000E5FFFFFF9D
:1046B0000A6802F8010B0A60704710B5436913B12C
:1046C000AFF3008001E0FFF706FE012010BD127875
:1046D00000F124010A7000224A700122EDE71168FE
:1046E0004FF0FF32E9E7754600F028F8AE460500C6
:1046F0006946534620F00700854618B020B5FEF7FE
:10470000D7FFBDE820404FF000064FF000074FF004
:1047100000084FF0000B21F00701AC46ACE8C009DF
:10472000ACE8C009ACE8C009ACE8C0098D467047E8
:104730000446AFF300802046FBF729FD0048704790
:10474000580100207047000001491820ABBEFEE769
:104750002600020030380A2801D2012070470020CC
:104760007047000000000000000000000000000092
:104770000404040404040004000000140A0A0000F5
:10478000000000000000000014143F140A3F0A0A51
:10479000000000041E1505060C14150F040000008F
:1047A00012150D0A142C2A1200000000040A0A1E19
:1047B000151509360000000202010000000000008B
:1047C0000000002010080808080808102000000257
:1047D0000408080808080804020000000004150E78
:1047E0000E150400000000000404041F040404006B
:1047F00000000000000000000000000202010000B4
:104800000000001F00000000000000000000000089
:104810000000000200000010080808040402020260
:10482000010000000E1111111111110E0000000005
:10483000040604040404040E000000000E11110814
:104840000402011F000000000E11100C1010110EC8
:1048500000000000080C0A0A091E081800000000E9
:104860001F01010F1010110E000000000E09010FB2
:104870001111110E000000001F09080404040404B3
:10488000000000000E11110E1111110E00000000A9
:104890000E1111111E10120E000000000000040085
:1048A00000000004000000000000000400000004FC
:1048B000040000201008040204081020000000007A
:1048C00000001F00001F000000000002040810206C
:1048D00010080402000000000E1111080404000476
:1048E000000000000E111915151D011E000000002A
:1048F00004040C0A0A1E1233000000000F12120EEC
:104900001212120F000000001E1101010101110E10
:10491000000000000F1212121212120F000000000D
:104920001F120A0E0A02121F000000001F120A0EB8
:104930000A020207000000001C1201013911120CCA
:10494000000000003312121E121212330000000089
:104950001F0404040404041F000000003E080808AB
:10496000080808090700000037120A060A0A123769
:1049700000000000070202020202223F00000000C5
:104980001B1B1B1B15151515000000003B121616EE
:104990001A1A1217000000000E1111111111110E38
:1049A000000000000F12120E0202020700000000B9
:1049B0000E1111111117190E180000000F12120E0E
:1049C0000A121237000000001E1101060810110F14
:1049D000000000001F1504040404040E0000000081
:1049E000331212121212120C000000003312120ABB
:1049F0000A0C0404000000001515150E0A0A0A0A24
:104A0000000000001B0A0A04040A0A1B0000000040
:104A10001B0A0A040404040E000000001F09080415
:104A20000402121F0000001C040404040404040413
:104A30001C00000202020404080808100000000E16
:104A400008080808080808080E0000040A0000000A
:104A50000000000000000000000000000000000056
:104A6000003F000400000000000000000000000003
:104A70000000000C121C123C000000000302020E99
:104A80001212120E000000000000001C1202021C94
:104A9000000000001810101C1212123C0000000050
:104AA0000000000C121E021C000000003804041E4E
:104AB0000404041E000000000000003C120C021E52
:104AC000221C00000302020E121212370000000026
:104AD000040000060404040E000000000800000C9E
:104AE00008080808080700000302023A0A0E1237F5
:104AF00000000000070404040404041F0000000078
:104B00000000000F15151515000000000000000F33
:104B100012121237000000000000000C1212120CDA
:104B2000000000000000000F1212120E0207000029
:104B30000000001C1212121C103800000000001BA4
:104B400006020207000000000000001E020C101EFA
:104B5000000000000004040E04040418000000001B
:104B60000000001B1212123C000000000000003781
:104B7000120A0C040000000000000015150E0A0ABD
:104B8000000000000000001B0A040A1B00000000D7
:104B900000000037120A0C04040300000000001E8D
:104BA0000804041E00000018080808040808080883
:104BB0001800080808080808080808080808000677
:104BC000040404080404040406000225180000007C
:104BD00000000000000000000000000000000000D5
:104BE000000000000000000000080808080808088D
:104BF00000001818000000486C241200000000009B
:104C00000000000000000000002424247F12121283
:104C10007F12121200000000081C2A2A0A0C182811
:104C2000282A2A1C080800000022251515152A58D4
:104C30005454542200000000000C1212120A76256F
:104C40002911916E00000006060403000000000018
:104C500000000000000000402010100808080808AC
:104C60000810102040000002040808101010101056
:104C70001008080402000000000008086B1C1C6BF0
:104C800008080000000000000000080808087F086D
:104C900008080800000000000000000000000000FC
:104CA0000000060604030000000000000000FE00F3
:104CB00000000000000000000000000000000000F4
:104CC0000000060600000000804040202010100870
:104CD000080404020200000000182442424242423A
:104CE000424224180000000000080E0808080808C6
:104CF0000808083E00000000003C4242422020100C
:104D00000804427E00000000003C4242201820407F
:104D10004042221C000000000020302824242222CF
:104D20007E20207800000000007E0202021A264049
:104D30004042221C0000000000382402021A2642D1
:104D40004242241800000000007E222210100808B1
:104D50000808080800000000003C424242241824D1
:104D60004242423C00000000001824424242645883
:104D70004040241C00000000000000001818000043
:104D800000001818000000000000000000080000EB
:104D9000000000080804000000402010080402047D
:104DA0000810204000000000000000007F0000000C
:104DB0007F000000000000000002040810204020D6
:104DC0001008040200000000003C4242464020104F
:104DD0001000181800000000001C225A55555555A7
:104DE0002D42221C00000000000808181414243C66
:104DF000224242E700000000001F2222221E22421F
:104E00004242221F00000000007C424201010101D9
:104E10000142221C00000000001F22424242424286
:104E20004242221F00000000003F4212121E1212D6
:104E30000242423F00000000003F4212121E1212C6
:104E40000202020700000000003C22220101017161
:104E50002122221C0000000000E7424242427E4222
:104E6000424242E700000000003E08080808080827
:104E70000808083E00000000007C10101010101000
:104E800010101010110F0000007722120A0E0A12E3
:104E90001222227700000000000702020202020232
:104EA0000202427F000000000077363636362A2A9A
:104EB0002A2A2A6B0000000000E346464A4A525262
:104EC0005262624700000000001C22414141414102
:104ED0004141221C00000000003F424242423E028B
:104EE0000202020700000000001C22414141414132
:104EF0004D53321C60000000003F4242423E1212FD
:104F0000222242C700000000007C42420204182016
:104F10004042423E00000000007F4908080808089F
:104F20000808081C0000000000E7424242424242DA
:104F30004242423C0000000000E742422224241486
:104F40001418080800000000006B494949495555EC
:104F5000362222220000000000E7422424181818FC
:104F6000242442E7000000000077222214140808DD
:104F70000808081C00000000007E21201010080412
:104F80000442423F000000780808080808080808A2
:104F90000808080878000000020204040808081045
:104FA000102020204040001E101010101010101073
:104FB000101010101E000038440000000000000017
:104FC00000000000000000000000000000000000E1
:104FD0000000000000FF00060800000000000000C4
:104FE000000000000000000000000000003C4278CB
:104FF000444242FC0000000000030202021A264262
:105000004242261A0000000000000000003844025E
:1050100002024438000000000060404040784442F2
:10502000424264D80000000000000000003C427EC4
:105030000202423C0000000000F08808087E0808D8
:105040000808083E0000000000000000007C22224A
:105050001C023C42423C000000030202023A46426B
:10506000424242E700000000000C0C00000E08085D
:105070000808083E00000000003030000038202002
:1050800020202020221E0000000302020272120AC9
:105090001612227700000000000E08080808080811
:1050A0000808083E0000000000000000007F929207
:1050B000929292B70000000000000000003B4642C0
:1050C000424242E70000000000000000003C424273
:1050D0004242423C0000000000000000001B26424B
:1050E0004242221E020700000000000000784442F5
:1050F0004242447840E000000000000000774C0489
:105100000404041F0000000000000000007C4202B4
:105110003C40423E0000000000000008083E080835
:105120000808083000000000000000000063424250
:10513000424262DC000000000000000000E7422460
:1051400024140808000000000000000000EB49499A
:1051500055552222000000000000000000762418AF
:105160001818246E000000000000000000E7422430
:10517000241418080807000000000000007E221018
:105180000808447E000000C020202020201020209D
:1051900020202020C000101010101010101010102F
:1051A0001010101010100006080808080810080851
:1051B0000808080806000C32C200000000000000C9
:1051C000000000000000C9EE000027FC140414A435
:1051D000811042084040104017FC2040E0E0215080
:1051E00022482C4620400040DBDA1104112411240F
:1051F00011241124FD24112411241124112411241B
:105200001D24E124422402040404CAD00200010047
:1052100000007FFC0100010001003FF82108210887
:10522000210821082128211001000100C8AB00003D
:105230000000018002400430180860061FF90100D8
:10524000010001003FF80100010001007FFEB6AF40
:105250000000000000203E20007C002200227F226F
:105260001022102212221222224223423D82009C4E
:10527000B5E70000010001001FF0610C410441048A
:105280007FFC4104410441047FFC01000102010252
:1052900001FCD7D3000000003FF800100060008040
:1052A000010000807FFE0040004000200020002020
:1052B00018400780BCBC10201020102013FEFC20DA
:1052C0001020102015FC18843088D0481050102071
:1052D000105051882606CAF5010001200110011066
:1052E0007FFC03800540054009201110210841047E
:1052F0008102010001000100D3D002000200FFFE84
:10530000040004000FF0081018102FF04810881047
:105310000FF00810081008500820CFDE00007BF8BE
:105320004A08520853F8620852084BF84A444A485F
:105330006A3052204210428843064200B9AB0080D6
:105340000480048008400840102020104208820693
:1053500004000440082010203FF010100000CBBED5
:1053600000003FF8000800087FE8000800081F88D8
:1053700010881088108810881F8810880028001056
:10538000BBB600800080FC8004FC050449082A406C
:105390001440104028A024A04510811002080404E5
:1053A0000802D3AD00002080133C12240224022402
:1053B000F2241224122412B41328122010202820C0
:1053C00047FE0000C4FA0900090011FC32045448E9
:1053D00099501148124414441140108002005104A5
:1053E000511290120FF0B4BF00000020102013FEE5
:1053F000202026244A247A241224222423FC7C20E0
:10540000002204227822003CC9AB00000000040006
:105410000FF0102020207FFC208420842084208412
:105420003FF82000200220021FFECCEE000000000A
:10543000204023FE204079FC220423FC220423FC8C
:10544000220423FC3A0465FA01980204B3E4000044
:10545000010001007FFE02200410040808043FFC44
:10546000044204400440044208421042607EBED818
:1054700000000000207E3E804880488048FE488230
:105480007F8208820C8214FA12842280218040FEDE
:10549000D0CE000000007F842208223022C02202E9
:1054A00022047FC8223022C2220222042208223093
:1054B0004040BBAD000000007FFE00000FF0111067
:1054C0001110111051125FF25112511251124FF27C
:1054D00040027FFCD4B2000000007FFE47E2481289
:1054E000481247E24FF2501250125112511242929A
:1054F0004472580A3FFCCDBC000000003FFE44024D
:1055000047F24C225362408243625E1A41824062FB
:10551000430240C240223FFCC6AC00000040204095
:10552000204020403FFE2000200020003FE02010CF
:1055300020102010201040104010CFD40000000098
:105540003FFC200420043FFC200420041FF82444D6
:105550001448144814480C5004407FFECABE000092
:1055600000003FFC0000000000007FFE008008906B
:105570000888108810842084208240820780B2CB63
:105580000000002008207FFE002000783F881108DE
:10559000089009207FFE018003400D30310C40024D
:1055A000B5A500000010081004203FF821042104D4
:1055B0003FFC210421043FF801007FFE01000100AF
:1055C0000100D6D000000100010001003FFC2104D1
:1055D000210421042104210421043FFC01000100D5
:1055E00001000100D3A20000000008207FFE082077
:1055F000092001003FF82108210821081FF401407B
:1056000002200C10700ECEC40000010001000080CA
:105610003F7C081008100410042002200240018082
:10562000018002601C18E006D7DB0000000010209B
:1056300011FE2202220249FC5800300013FE2528E8
:10564000792401240D24722202A2BACF00000000A6
:10565000018002400430180860061FF800001FF89F
:10566000200420042004200420041FF8C1C10000ED
:10567000010001007FFE00003FF820083FF83FF8DE
:10568000400647C24824082008221022603EB6C8BF
:105690000000000000803FFE44105FFC44104410F6
:1056A00043F040005FF84408423041C04360BC1EF4
:1056B000B2E20000000067C2145205520552C55202
:1056C0002552055205521552175222822242444257
:1056D000483ECAD4000000002014101417FE001227
:1056E0000010601013F0109010901090149214EAB3
:1056F0001F0A0006B3CC0000000019FE720212025D
:1057000012027DFC18001BFE3420502053FE102096
:105710001020102013FED0F20000000000803FFE99
:10572000400047FC4208413040C05FFE40424042DA
:105730004044404840404440B5F70000000023FE8C
:10574000122202FA0222E22212FE1272128A128A35
:10575000128A16BA1A421202040EB9E200000100BF
:10576000010411080908091009207FFE04400440C3
:1057700004400440084208421042607CB0E6000049
:10578000000048FE4900490049007EFE4182414434
:105790007944452845284510452846440382C8A831
:1057A00000001000100013FC7D041104190418847B
:1057B00034885048505010201050108813041402A0
:1057C000CBF9000000003F7C204020403E40227E7C
:1057D0002244224422443E84208420844084410484
:1057E0004204C6C100003FF8200820083FF82410FA
:1057F00022202FF8222022203FFC22204220442079
:1058000084200820C4BB04407FFC04401FF010101B
:105810001FF010101FF00400FFFE11103FF8D1160A
:10582000115011200100D0FD2080108010FE0100D9
:10583000FE0021FC20243C2424A024A024BC24A07D
:1058400024A04560553E8A00D7AA20202020202091
:10585000FDFC4020504093FEFC40108011FC1C04D5
:10586000F0885050102010101010BFAA00007FFCCC
:1058700008200820082008200820FFFE0820082013
:10588000082008201020102020204020D4B4000040
:1058900027FE1420144085FC450445FC150415FC26
:1058A0002524E42024A829242A2230A00040D2BAAA
:1058B0000080204017FE11208120423C42441664A3
:1058C00012942348E24822302220225022880306E4
:1058D000BEA70FE0082008200FE0082008200FE0F6
:1058E00000007EFC428442847EFC428442847EFC32
:1058F0004284CDF800007FFC4004400442145294DE
:105900004A54442444244A544A545294610440045E
:1059100040144008D5BE1020082008207E20003EFC
:1059200004204420442025FC290429040F04F10408
:10593000410401FC0104B0B410401020102013FEFB
:10594000FA02144410401BFE3088D088110810D091
:105950001020105050882304BCFC201020103B7CE9
:10596000211441FE7A14A27C2710F97C251025FE13
:1059700022102A10350028FE0000D0A3104010206D
:10598000102011FEFC00108831043A02548850881F
:10599000905010501020105010881306D7BC0140B2
:1059A0004120212023FE022016201BFC1220222051
:1059B00023FCE2202220222023FE22000200B4A5A4
:1059C00020202020782049FC91247D245524552432
:1059D0007DFC552454207C28542457FE45028C001D
:1059E000C3FE1110111017FC1110FC0013F812085F
:1059F00017F81A0833F8D04017FC10A011105208FD
:105A00002406B6C10020202011FC1020002003FE37
:105A1000F002109410501110109013FE1428184426
:105A200010820302BACD04000E007800087C0844FE
:105A3000FF44084418441C442A442A444844887CAF
:105A4000084408000800D1D5100008FE7F1022206D
:105A5000147C7F4444544854525444544854515440
:105A60004228442488423082D6B5084008400FFCC2
:105A70001040104033F8320853F8920813F8120817
:105A800013F8120812081FFE1000C8DD0200010002
:105A90007FFE40028824111022880440082030181C
:105AA000DFF61010101010101FF01010D6A7010014
:105AB000010001007FFC0100010001003FF0101017
:105AC000082004400280010006C01830E00EB3D662
:105AD00010201020102011FCFC20102013FE1008B4
:105AE000180833FED00810881048100850282010DD
:105AF000B5E302000200020003FC020002003FF0D6
:105B00002010201020103FF000002488224442443E
:105B10008004CCAC010001007FFC01000280044045
:105B20000A203118C006010008884884481248122B
:105B300087F00000CAFD082049202A20083EFF44C3
:105B40002A44494488A41028FE28221042106428C0
:105B500018283444C282D7D6020001007FFE4002DA
:105B600080041FE0004000800100FFFE01000100F2
:105B70000100010005000200CDCB03F82208120845
:105B800013F802080208F3F81244122812101288BF
:105B900013041204280047FE0000B3F601000100C0
:105BA00021082108210821083FF80108010001000F
:105BB00041044104410441047FFC0004C9EE00009B
:105BC000000000001000000800080C7FFC044010DA
:105BD00001C8A002186042301832231812C3001402
:105BE000030004030C047FF0080F80080B407813B7
:105BF0006018332018631818831C19030818030051
:105C0000000300000000DBDA0000000000000410C8
:105C10000C04180C04108C04108C04108C04108CD0
:105C200004D08C3F108C04108C04108C04108C0455
:105C3000108C04108C04108C05F08C0E208C7820B5
:105C40008C20408C00808C01000C02000C000000B5
:105C5000CAD000000000000000300000180000184A
:105C60000800001C1FFFE000180000182007FFF0CC
:105C700004182004182004182004182004182004F4
:105C800018200418200418200418200418E0041810
:105C900040001800001800000000D6D000000000EE
:105CA00000000000000000000018000018000018AC
:105CB000000018003FFFFE301806301806301806A6
:105CC0003018063018063FFFFE3018060018000096
:105CD0001800001800001800001800000000000064
:105CE00000000000CEC40000000000000000000022
:105CF0003800001C00000600FFFFFF060030060011
:105D0000300300600300600180C000C18000E30038
:105D1000003600001C0000770003C1E01E003C605C
:105D20000007000000000000000000000000B2E2D8
:105D300000000000000000000000000040000321FF
:105D4000FF33398333118333019B33C19B33719B01
:105D500033199B33019B33019B33119B3319B333AD
:105D6000303033306C0330C6036383032E01BE0032
:105D70000000000000000000CAD400000000000085
:105D80000000000000004000D83000CE1800C21C07
:105D900000C001FFFF0000C0F800C01800C019FFDC
:105DA000C01818401818601918601B18611E1831A7
:105DB0001C1FB139F01910000F0000000000000096
:105DC0000000D7D60000000000060000000300001D
:105DD0000000C0000001C0C0000107C00001FF00BA
:105DE000021FFE0007F01C0007C070000F00E0005B
:105DF0000E03F0001C0FF0003C0F70003C00E000B0
:105E00001800C0000000C0000000C00000006000DA
:105E100000002000000037000001FF00007FF800B4
:105E200007F830001F8030000080300000C03000D4
:105E3000006060000018E000000FC00000060000D5
:105E400000000000CCE500000000000000000000A1
:105E500000C0000000E0002001B800703FF80061C1
:105E6000FFC000C3030001C60600038C0600030840
:105E70000C0006080C000E18183F1E101BF31F9094
:105E80003F0700803C1C0190707C019060FE01A0E7
:105E9000C3F801A00FD803A008180360001803403E
:105EA000001803C000180380001803000018000049
:105EB000001800000010000000300000003000005A
:105EC000000000000000B2E200000000000000003E
:105ED0000000000000000000020C1008071FF8047A
:105EE00003BFF00201BC300303EC3003015C60032C
:105EF00000D8600300D860038098620361B843074C
:105F000071B14306313243063376C3063A64C7069D
:105F10003EECC0063E78C0063C3040067C70000671
:105F200078E060067BFFF006F7C00006E40000069C
:105F300040000006000000060000007C00008FF01A
:105F400000007C0000000000CAD400000000000037
:105F500000000000000000003F0000007F80000003
:105F60000180000000C0000000C0000000CE0380DF
:105F700000CFFFC000DD41800FFE0007FFFC000CDA
:105F800000F000180FC03E19FF40F311BC608330D1
:105F90007FE003B1FE2003338020037000300360F4
:105FA00000100360001807C0000C07C00004078041
:105FB00000020100000300000001000000000000DA
:105FC000000000000000000000000000FFFFFFFFD5
:105FD000FFFFFFFFFFFFFFFFFFFFFFFFFFFFFFFFD1
:105FE000FFFFFFFFFFFFFFFFFFFFBEF7FFFFDEFF2B
:105FF00038C6928C8E6B6E6B107C96AD3CE7FFFFC3
:10600000FFFFFFFFFFFFFFFFFFFFFFFFFFFFFFFFA0
:10601000FFFFFFFFFFFFFFFFFFFFFFFFFFFFFFFF90
:10602000FFFFFFFFFFFFFFFFFFFFFFFFFFFFFFFF80
:10603000FFFFFFFFFFFFFFFFFFFF5DEF159D4F63BA
:106040006C420A328829461925194521E8318E6BA0
:1060500038C6FFFFFFFFFFFFFFFFFFFFFFFFFFFF50
:10606000FFFFFFFFFFFFFFFFFFFFFFFFFFFFFFFF40
:10607000FFFFFFFFFFFFFFFFFFFFFFFFFFFFFFFF30
:10608000FFFFFFFFFFFFFFFF36A51053104B5153DB
:106090000F4B6C3AE93167212519E410A30862001F
:1060A0008308CB529AD6FFFFFFFFFFFFFFFFFFFFE2
:1060B000FFFFFFFFFFFFFFFFFFFFFFFFFFFFFFFFF0
:1060C000FFFFFFFFFFFFFFFFFFFFFFFFFFFFFFFFE0
:1060D000FFFFFFFF3CE77063B363B87CF5631143D8
:1060E0004D32EA29882126190519051904110411D0
:1060F000E4108300A308728CFFFFFFFFFFFFFFFF88
:10610000FFFFFFFFFFFFFFFFFFFFFFFFFFFFFFFF9F
:10611000FFFFFFFFFFFFFFFFFFFFFFFFFFFFFFFF8F
:10612000FFFFDBDE4B3AF042356C544BB1322E2A86
:10613000EB21A92167190519041104110411041197
:1061400004110519E4104200AF73FFFFFFFFFFFFCA
:10615000FFFFFFFFFFFFFFFFFFFFFFFFFFFFFFFF4F
:10616000FFFFFFFFFFFFFFFFFFFFFFFFFFFFFFFF3F
:106170005DEF09324C32104B8F324F2A2E2ACC1948
:10618000891989214719051904110411C410C41073
:10619000041104110411E41042003184FFFFFFFFD9
:1061A000FFFFFFFFFFFFFFFFFFFFFFFFFFFFFFFFFF
:1061B000FFFFFFFFFFFFFFFFFFFFFFFFFFFFFFFFEF
:1061C000EC5247194C320B2AEC21EC210C22915B4A
:1061D000EE4A061126190419E410E410A7296621D5
:1061E000A308051904110411E4108200F7BDFFFF94
:1061F000FFFFFFFFFFFFFFFFFFFFFFFFFFFFFFFFAF
:10620000FFFFFFFFFFFFFFFFFFFFFFFFFFFF35A5C2
:106210008308882188218921AA218A216B42718CD7
:10622000FFFF728C83080411C4082942FBDE5DEF76
:10623000EC5A83080411041104118308E831DFFFCC
:10624000FFFFFFFFFFFFFFFFFFFFFFFFFFFFFFFF5E
:10625000FFFFFFFFFFFFFFFFFFFFFFFFBEF7C7319D
:10626000C4102519261947194719A8298A52284AFE
:1062700055ADFFFFE831A30805194D6B4D6BFFFFCE
:106280007DEF4521C410041104110411620076ADA4
:10629000FFFFFFFFFFFFFFFFFFFFFFFFFFFFFFFF0E
:1062A000FFFFFFFFFFFFFFFFFFFFFFFF96B562004D
:1062B0000411041905110519C4088B4AB6B55DEF20
:1062C000F7BDFFFF8E6B62002942AA5A0842FFFF0A
:1062D000FFFFCC528308041104110411A308AD522E
:1062E000FFFFFFFFFFFFFFFFFFFFFFFFFFFFFFFFBE
:1062F000FFFF1CE7FFFFFFFFFFFFFFFF4E63620092
:10630000041104110411E41062008E63FFFFFFFF0B
:10631000FFFFFFFFCF730100F39C2C6396B5FFFFD7
:10632000FFFF2D5B8300041104110411E4106721A9
:106330003DEFFFFFFFFFFFFFFFFFFFFFF8BDB7B51A
:106340009EEFCB52B394FFFFFFFFDFFFE831A308BE
:106350000411041104110411A3084942FFF7FFF7C7
:10636000FFFFFFFF6A4A01007284FFFFFFFFFFF794
:10637000DFEF093AA30804110411041104110511F7
:1063800018BEFFFFFFFFFFFFFFFFFFFFF07B620074
:10639000E831C731410035A5FFFF5DEF4621C4104C
:1063A0000411041104110411E410A308769DFFF7F1
:1063B000FFFFB7ADA308A308C7319EE7FFF7FFF7BC
:1063C00076A5A308E41004110411041105110511A8
:1063D00035A5FFFFFFFFFFFFFFFFFFFFDBDEA72964
:1063E0008300C410C410C4101CE79EEF0511E41014
:1063F00004110411041104110419C408E510D16B2F
:10640000D16BC5086400A50843002B32779DB38487
:106410002519C410041104110411041125192609A9
:10642000359DFFFFFFFFFFFFFFFFFFFFFFFFAF7384
:1064300062000419051982000D5B8E9B6210051124
:10644000041104110419E41085000511C439815A9E
:10645000407B229C43AC03A4839B82728249C21876
:10646000A400C500E41004190411051947196711A7
:10647000EC5ABEFFFFFFFFFFFFFFFFFFDFFFDBDE8A
:10648000C410E41004110511A41801C08388E400AD
:1064900005190419C5084421438323D542FEE4FEAF
:1064A00027FF07FFA4FE64FE03FEA3FDE2FC42EC0F
:1064B00083B32462E510C40804192619A81987219A
:1064C0000090D3BCFFFFFFFFFFFFFFFFDFFFFFFFD9
:1064D000107C420005190511832801D044F8A34817
:1064E000E400C508445A02EDE2FD02FE66FE74FFB8
:1064F000B8FF73FFE7F6A6F645F6A4F5C3FC62FC09
:10650000C2FCC2FCE3CBC449061188198701A490E0
:1065100001F8EC9AFFFFFFFFFFFFFFFFFFFFFFFF08
:10652000BEF7E83183000509824001C023F885F0F9
:10653000A348A400445A02FD23CCC2DC04FE28FE7A
:1065400048F646F624F6E4F564FDE3FC62FCC2FC82
:1065500002E402DCE2FCA47A48016701C47824F872
:1065600002F884B07DE7FFFFFFFFFFFFFFFFFFFFA3
:10657000FFFFDBDE2519A300C43802E022D844F86F
:10658000A6F8A4786300432183728339829B21F5A6
:1065900061FD22FDE2FCA2FC42FC42FC42FC22AB7B
:1065A0008341C392045226012519A49844F823F884
:1065B00002F8A4D09EEFFFFFFFFFFFFFFFFFFFFFEA
:1065C000FFFFFFFF9AD68729A50043B822F823E0F2
:1065D00065F8E8F807C983484200A30084006329EE
:1065E000A27A62B3A2CB62D302BB828A8339A400AF
:1065F000E500E500E508C46064D844F824F823F811
:1066000002F88388DBC6FFFFFFFFFFFFFFFFFFFFEE
:10661000FFFFFFFFFFFF3DE7505B083123E843F832
:1066200044F065F809F9ABF989D10689A348421805
:106630000200420061008200620062008300A32029
:10664000C450A58885D865F844F844F823F823F8A1
:1066500003D08210C7295DEFFFFFFFFFFFFFFFFFA1
:10666000FFFFFFFFFFFFFFFFFFFF6C32A53802D8DF
:1066700023F865F866F8A7F84AF90CFA4DFA4CEADF
:106680000BD2A9B968B147A927B107B907D1E7E883
:10669000C7F8A7F865F865F844F823F803F802D0BE
:1066A000A3280509C408EC5AFFFFFFFFFFFFFFFF07
:1066B000FFFFFFFFFFFFFFFFFBDE0519C400A7413F
:1066C000E6C003F886F8A7F887F886F8C7F829F92E
:1066D0008AF9ABF9ABF98BF96AF929F908F9C7F826
:1066E000A6F886F865F864F823F802F006B12529C3
:1066F000E400E41025192519149DFFFFFFFFFFFF9B
:10670000FFFFFFFFFFFFFFFF96AD62008208359598
:10671000BACE8BA244D025F887F8A7F8C7F8A7F817
:1067200087F886F886F886F887F8A7F8A7F8A6F815
:1067300085F865F864F824F064B80D93BBB6CF63B0
:1067400083080411E4106621493A5DEFFFFFFFFF63
:10675000FFFFFFFFFFFFFFFFD3944200E410BBCE1B
:10676000FFFFBEE776B5CCAA07C145E045F846F87D
:1067700066F886F886F886F886F865F845F865F8CC
:1067800065E844D043A8018882903CD7FFEF559537
:1067900083080411041105194619B394FFFFFFFF84
:1067A000FFFFFFFFFFFFFFFFB394410086215DDF86
:1067B000FFFFFFFFFFFFDFE77AC6D3B44EB32AC265
:1067C00068D1E6E0A6E8A5E8A5E8E6D888C906A964
:1067D00022A802A800A000C800D8F7E5FFE7F8AD9E
:1067E000C410E4100411E41005118B4AFFFFFFFFF1
:1067F000FFFFFFFFFFFFFFFF55A54100A7295DDF5A
:10680000FFF7FFFFFFFFFFFFFFFFFFFFFFEF7DDF52
:10681000DBCE59CEF8CDD7CDF7C579CEFBBEABA236
:1068200003F045F842D043E800F072D4FFDF39AE00
:10683000E410E4100411E41005118729FFFFFFFFA5
:10684000FFFFFFFFFFFFFFFF59CE830846211CD744
:10685000FFF7FFFFFFFFFFFFFFFFFFFFFFFFFFFF50
:10686000FFFFFFFFFFFFFFFFFFFFFFFFFFEF8BBA01
:1068700004F845F862E044F000F88EDBFFDFF8A58D
:10688000C410E410E4100411E4102519FFFFFFFF09
:10689000FFFFFFFFFFFFFFFFBEF78729830839B621
:1068A000FFF7DFF7FFFFFFFFFFFFFFFFFFFFFFFF28
:1068B000FFFFFFFFFFFFFFFFFFFFFFFFBEE74ABA3B
:1068C00003F845F864F844F800F86EE3FFD7F48C59
:1068D00083080411E410E410E4100519FFFFFFFF22
:1068E000FFFFFFFFFFFFFFFFFFFFEF73000072845A
:1068F000FFEFBEEFDFFFFFFFFFFFFFFFFFFFFFFF29
:10690000FFFFFFFFFFFFFFFFFFFFFFFFDFE78BBA88
:1069100003F845F845F823F800F8D3D4FFD74E5BC9
:106920002100293A55A58308C4102519FFFFFFFF50
:10693000FFFFFFFFFFFFFFFFFFFFFBDEA308E831C4
:106940009EDF9EE7BFEFFFFFFFFFFFFFFFFFFFFFA1
:10695000FFFFFFFFFFFFFFFFFFFFFFFFFFF751BC40
:1069600002E003F803F043E0ECC27ECFFCBE462118
:106970002100D394FFFF518400008729FFFFFFFF10
:10698000FFFFFFFFFFFFFFFFFFFFFFFF518400003E
:10699000F48CFFEF9EE7BFEFDFFFFFFFFFFFFFFF7E
:1069A000FFFFFFFFFFFFFFFFFFFFFFFFFFFF3DDFD9
:1069B00055BD52BC72BCB7B55DC7FFDFF06B0000C0
:1069C000093ABFF7FFFFFFFF149D55A5FFFFFFFF2B
:1069D000FFFFFFFFFFFFFFFFFFFFFFFFFFFFAC4ACF
:1069E000A408BBBEDFE77EE7BEEFDFF7DFFFFFFFF8
:1069F000FFFFFFFFFFFFFFFFFFFFFFFFDFFFDFF7EF
:106A0000FFEFDFDFBFD79ED7DFDFD8A583082611D2
:106A1000DBD6FFFFFFFFFFFFFFFFFFFFFFFFFFFFD3
:106A2000FFFFFFFFFFFFFFFFFFFFFFFF79EE8BDCA4
:106A30002131A9213DCFBFDF7EDF9EE7BEEFBFEF53
:106A4000DFF7DFF7DFF7DFF7DFF7BFEFBEEF9EE738
:106A50007EDF5ED75ED7DFDF9AB626194208EDA348
:106A6000BFFFFFFFFFFFFFFFFFFFFFFFFFFFFFFF76
:106A7000FFFFFFFFFFFFFFFFFFFF74DDC0DB00FE36
:106A800042EE024289217BB6DFDF7ED77EDF7EDFEA
:106A90009EE79EE79EE79EE79EE77EDF7EDF5DD76F
:106AA0005DD79EDFFFE7F8A50711E31802C560FD7B
:106AB000E6D3DBEEFFFFFFFFFFFFFFFFFFFFFFFF60
:106AC000FFFFFFFFFFFFFFFF9EF784BAC1FC42FEFE
:106AD00082FEA2FE8183452174745EC7DFDF7ED70C
:106AE0005ED75DD75ED75ED75DD75DD75ED79EDFB9
:106AF000FFE73DC7F1638408425226E629FF86FE80
:106B0000E0F36AC3FFFFFFFFFFFFFFFFFFFFFFFF91
:106B1000FFFFFFFFFFFFFFFF18DEC1D2A2FD22FE35
:106B200042FE42FE62FEE2D4416A494253743BA6F1
:106B30003EC7BFD7BFD7BFD7BFDFBFD73EC71AA695
:106B4000F263A729824122B462FE83FEAAFE0FFFF0
:106B500067FD63BA3CEFFFFFFFFFFFFFFFFFFFFF93
:106B6000FFFFFFFFFFFFFFFF9AE680D221FDC2FD7E
:106B7000E2F5C2F582F582FD62FD61DC219B846A4B
:106B8000E96A2C63AF6311746E632C63895A0452F3
:106B9000817AC2CBE2FC62FD82FDC2FDC2FDE4FD52
:106BA00024FD62CA1CE7FFFFFFFFFFFFFFFFFFFF9F
:106BB000FFFFFFFFFFFFFFFFFFFFB1CC81D2C0F35C
:106BC000C1FC02FD02FDE2FCC2FCC2FC81FC80FBB8
:106BD000C0C9A48135AD59CE719C218100DAA1FBD9
:106BE00082FCA2FC82FCA2FC02FD22FDE2FC00FC75
:106BF00060DA90CCFFFFFFFFFFFFFFFFFFFFFFFF0B
:106C0000FFFFFFFFFFFFFFFFFFFFFFFF59DE0DC488
:106C100006CBE4D203DB03DBE3DAC3D2A4C209B3BD
:106C2000D2BC9EF7FFFFFFFFFFFFFBE60EB4A6BA44
:106C300083D2E3E202EB22EB22E303DBE4D26AC37A
:106C4000B6D5FFFFFFFFFFFFFFFFFFFF00F80000CB
:106C5000CC6C0008C06C0008B06C0008A06C000888
:106C60000300090030313233343536373839414288
:106C7000434445464030580030313233343536379E
:106C8000383961626364656640307800040000084A
:106C900000000000000000020001000010000000E1
:106CA000526F746174696F6E3A32373000000000C1
:106CB000526F746174696F6E3A31383000000000B1
:106CC000526F746174696F6E3A393000526F74613B
:106CD00074696F6E3A300000F86C00080000002004
:106CE00064000000280100085C6D000864000020BA
:106CF000540300004401000800A24A040000000000
:106D000000000000010203040607080900F8E0077C
:106D10001F00E0FF1FF800F81FF8E007CF011F0079
:106D200000001F8400000000FFFF0000A52F0008E6
:106D30000000000000000000000000000000000053
:106D4000000000000001020304010203040607081A
:0C6D50000902040608000000000000001A
:04000005080000ED02
:00000001FF
